:1064710001190000090101240200000301FA0400CE
:10648100FA0500030A0A5A0B001E0C00FA0D00035C
:106491000E00040F0164100096120132130AFA145F
:1064A100010215000217010A1801FA1905321A0131
:1064B1000A1B01FA1C05321FFFFF20FFFF23011EEB
:1064C1002400642A00FA2B00FA2C50782D003D2E6E
:1064D10000462F001E300064325078330000343201
:1064E100FA350164360164370150380A643C0064AE
:1064F1003E003C3F000140FFFF411450420A5A4315
:106501000AC84405324500B44600FA47014848022A
:10651100034C00FA4EFFFF500404510596520A3213
:10652100530B46540A965601025705465800025924
:106531000A465A32FA5B010A5C0A325E000A5F00BF
:10654100FE61FFFF64021066000267FFFF6A0A3CFA
:106551006B00006C32967300007400007801327990
:1065610001327EFFFF81FFFF84FFFF8500AF8600C0
:10657100018700FA89010A8A00009900009D0A96A4
:106581009E00019FFFFFA0FFFFFAFAFA0065006F6E
:1065910000790083008D009700A100AC00B600C017
:1065A10000CA00D400DE00E800F200580060006874
:1065B10000700078008000880090009800A000A87A
:1065C10000B000B800C100C800D000D800DF00E66C
:1065D10000EE00F600410047004D00530059005FF6
:1065E1000065006C00710077007D00830089008FD9
:1065F1000095009B00A200A700AC00B200B900C04A
:1066010000C500CA00D200D500DD00E100E700EFBF
:103A39009007BAE0FEA3E0FF90647312674AE4932B
:103A4900F599906471E493FC740193FDEFB5050752
:103A5900EEB50403754D009007BA1267312285F956
:103A69007385FA747E017F00E574126723E5732F6D
:103A7900FF50010E8E5A8F5B900013E0FCA3E0FD0E
:103A8900EF2DFDEE3CFC8C5C8D5D2275A71085F950
:103A99007385FA747E017F00E574126723E5732F3D
:103AA900FF50010E8E5A8F5B9000DCE0B40210AC1F
:103AB9002CAD2DEF2DFDEE3CFC8C5C8D5D8016AEA2
:103AC9005AAF5B900013E0FCA3E0FDEF2DFDEE3C47
:103AD900FC8C5C8D5D22AE5AAF5B740A8E048F0537
:103AE900FF1267138C5C8D5DAE5AAF5B740A8E044E
:103AF9008F05FF12673E8C5A8D5BE55B455A601353
:103B0900740AC3955BFFE4955AFE8E5A8F5B785C05
:103B1900126777E573A85CB80015D3955D4010E589
:103B290073C3955DFFE4955CFE8E5C8F5D8010E547
:103B3900732424C3955DFFE4955CFE8E5C8F5D75EF
:103B49007300AE5CAF5D74116F4E600674126F4EF8
:103B59007018AE5CAF5D74116F4E7005757301809E
:103B690003757302755D10755C00AE5CAF5D74140E
:103B79006F4E600674156F4E7018AE5CAF5D7414AD
:103B89006F4E70057573018003757302755D13754A
:103B99005C00AE5CAF5D74236F4E600674246F4E9B
:103BA9007018AE5CAF5D74236F4E7005757301803C
:103BB90003757302755D22755C002290008AE0B47A
:103BC9000104C2108002D21090008BE0B40104C23B
:103BD900118002D2119000C8E075F0DCA4FFAEF0AC
:103BE900740A8E048F05FF1267139007B0ECF0A3D7
:103BF900EDF0A20D401674038C068D07126723742D
:103C0900011200399007AEEEF0A3EFF07E017F00BC
:103C1900900086E01267239000C9E08E048F05FFAB
:103C2900126713740AFF1267138D609000D2E07552
:103C3900F0DCA4FFAEF0740A8E048F05FF1267133F
:103C49009007B4ECF0A3EDF09000D4E0601390007D
:103C5900D4E0F5F0741684FF7E00EF9007C2F0807F
:103C69000674649007C2F09000CAE090006EF0906C
:103C79000114E0900058F09000A3E090005AF090F1
:103C890000CCE090005BF0900078E090005CF09050
:103C990000FEE0900061F0900162E0900062F09017
:103CA9000163E0900063F0900164E0900064F0A289
:103CB90027B34016900162E0700C900163E0700632
:103CC900900164E060028002C22774E390006DF005
:103CD9009000B3E0B40B0874E390006DF0805A9043
:103CE90000B3E0B419129000C9E090657812008C15
:103CF900E49390006DF080419000B3E0B41E1290FF
:103D090000C9E090659612008CE49390006DF080F4
:103D1900289000B3E0B428129000C9E09065C01261
:103D2900008CE49390006DF0800F9000B3E0B446EE
:103D3900089000AAE090006DF09000E3E0FE90008A
:103D4900B1E06E600A9000B1E09000E3F0D22690F5
:103D59000071E0FE9000B0E0B50633900073E0FE1C
:103D69009000CEE0B50627900072E0FE9000DCE0FE
:103D7900B5061B900075E0FE900083E0B5060F9034
:103D89000074E0FE9000BEE06E7003023ED7900022
:103D990049E0C39405500874029000FFF080149024
:103DA90000DCE0600874089000FFF08006740A9057
:103DB90000FFF0900083E0B4010674009000E9F080
:103DC900900083E0B4020674009000CEF090008366
:103DD900E0B4030674009000DBF09000CEE0D394C9
:103DE9000140147418900101F074009006C8F07431
:103DF900009006C9F0800C7400900101F0741890CD
:103E090006C8F09000B0E06014741A900097F0743E
:103E1900009006D0F074009006D1F0800C740090E8
:103E29000097F0741A9006D0F09000B0E0B4021434
:103E39007419900098F074009006CCF07400900604
:103E4900CDF0800C7400900098F074199006CCF0B5
:103E59009000DCE0700E74059006DCF074069006A4
:103E6900E0F0801874009006DCF074009006DDF034
:103E790074009006E0F074009006E1F0D2269000FC
:103E8900B0E0900071F09000DCE0900072F09000DA
:103E9900CEE0900073F09000BEE0900074F09000C6
:103EA90083E0900075F0900083E0900059F0900055
:103EB900BEE090005DF09000DCE090005EF09000C4
:103EC900B0E090005FF09000CEE0900060F09000CC
:103ED900E6E0B4011790001F740FF0A374FFF0908F
:103EE9000021E4F0A3F074029000E6F09000E6E00F
:103EF900B40341900021E0FEA3E0FF90001FE0FC25
:103F0900A3E0FD12676F7410126723740812003959
:103F1900EF90006AF0EF700674FF90006AF0740089
:103F29009000E6F0900020E090006BF090001FE018
:103F390090006CF0900077E090003BF090003BE03F
:103F4900241290003CF090003CE0D39424400B9064
:103F5900003CE0C3942490003CF090003FE4F090D2
:103F6900003BE06411600790003BE0B41220900030
:103F79003BE0B41106740290003FF090003BE0B4BE
:103F8900120690003F7401F0741390003BF090000A
:103F99003BE06414600790003BE0B4152090003BBF
:103FA900E0B41406740290003FF090003BE0B415B1
:103FB9000690003F7401F0741690003BF090003BAE
:103FC900E06423600790003BE0B4242090003BE0CC
:103FD900B42306740290003FF090003BE0B424063D
:103FE90090003F7401F090003B7401F0900040E4B0
:103FF900F090003CE06411600790003CE0B41220AE
:1040090090003CE0B411067402900040F090003C2E
:10401900E0B412069000407401F0741390003CF073
:1040290090003CE06414600790003CE0B4152090D7
:10403900003CE0B414067402900040F090003CE0AB
:10404900B415069000407401F0741690003CF0908D
:10405900003CE06423600790003CE0B42420900019
:104069003CE0B423067402900040F090003CE0B4B8
:1040790024069000407401F090003C7401F0900017
:1040890077E0FE9000DAE02E900042F0900042E0E6
:1040990064036017900042E06412600F900042E0F0
:1040A90064156007900042E0B42406900042E004E1
:1040B900F0900042E064026017900042E0641160F1
:1040C9000F900042E064146007900042E0B42306B8
:1040D900900042E014F0900042E0D39424400B9009
:1040E9000042E0C39424900042F0900042E0D3944F
:1040F90012400D900042E0C39412900043F0800AF0
:10410900900042E02412900043F07551129000BDD6
:10411900E090003DF090003DE0B4020690003D744F
:1041290001F090003DE0B40306740490003DF09066
:10413900003DE0B41106741090003DF090003DE0A0
:10414900B41206741390003DF090003DE0B41406DB
:10415900741390003DF090003DE0B415067416907C
:10416900003DF090003DE0B42306742290003DF03C
:1041790090003DE0B42406742590003DF090003D88
:10418900E0B42606742590003DF090003DE0B42788
:1041990006742890003DF090003DE0B43506743473
:1041A90090003DF090003DE0B43606743790003D34
:1041B900F090003DE0B43806743790003DF090006F
:1041C9003DE0B43906743A90003DF090003DE0B40A
:1041D9004706744690003DF090003DE0B4480690D3
:1041E900003D7401F090003DE0D39424400F90000D
:1041F9003DE0C3942490003DF0D2208002C220907B
:10420900003DE0D39412400D90003DE0C39412901C
:10421900003EF0800A90003DE0241290003EF0221A
:10422900C293C294C291C292C287C290E5B554EFBB
:10423900F5B5E5B554DFF5B5C296C295C2A0C297EA
:10424900C2A2C2A1E5B554BFF5B5E5B5547FF5B530
:10425900E5B554FBF5B5C212755E469000C0E07035
:1042690005756D028003756D0375550075540090D1
:10427900000874FFF0A374DCF0C217C21974C89067
:104289000033F074C8900037F0755300755200C2BE
:104299000D754600E56FB40903756F0075630090ED
:1042A9000015E4F0A3F0757010C215C2169007B09E
:1042B900E0FEA3E0FF740312672374011200399032
:1042C90007AEEEF0A3EFF0C20275570075560090E5
:1042D900000CE4F0A3F0C22875590075580090004D
:1042E90082E075F032A4FDACF090001DECF0A3ED76
:1042F900F0C238A22CB39205A22DB39206A22EB316
:104309009207A22FB39208A230B39209A231B392B5
:104319000AA232B3920BA233B3920C2285F97385A8
:10432900FA747E017F00E574126723E5732FFF504D
:10433900010E8E5A8F5BAC5CAD5DEF2DFDEE3CFC42
:104349008C5C8D5DD293D294E55DF5FBE55CF5FC63
:10435900E55DF5E9E55CF5EA9000BEE0B40314D249
:1043690091D292E55DF5EBE55CF5ECE55DF5EDE502
:104379005CF5EE2275A71085F97385FA747E017FC5
:1043890000E574126723E5732FFF50010E8E5A8FD3
:104399005B7E017F769000FBE0126723AC5AAD5B30
:1043A900ED2FFFEC3EFE8E5C8F5DE55DF5FDE55C76
:1043B900F5FE90006EE4F075A7007412900045F0C8
:1043C9002285F97385FA747E017F00E574126723EB
:1043D900E5732FFF50010E8E5A8F5B9007B0E0FCFA
:1043E900A3E0FDEF2DFDEE3CFC8C5C8D5DE55DF5FC
:1043F900FDE55CF5FE220564229000BEE0B403539E
:104409009000DCE0B4012EA2D8B34004C293C28765
:10441900A2D9B34004C294C290A2DAB34008C291AF
:10442900E5B554EFF5B5A2DBB34008C292E5B55442
:10443900DFF5B5801CA2D8B34002C293A2D9B3401C
:1044490002C294A2DAB34002C291A2DBB34002C213
:1044590092801EA2D8B3400AC2939000DCE06002A9
:10446900C287A2D9B3400AC2949000DCE06002C2BC
:1044790090A2DCB34004C296C29575D8402285A7A4
:104489007275A710A2D8B34002C287A2D9B340025D
:10449900C290A2DAB34006E5B554EFF5B5A2DBB395
:1044A9004006E5B554DFF5B5A2DCB340089000CA73
:1044B900E090006EF075D8408572A722900047E41D
:1044C900936406600280FE74C89007B6F8E4F0E8C9
:1044D900A3F075B50075840175A70075FFA090005C
:1044E90041E4F075C91075A70F75A1C775A70075C7
:1044F900D90075CE0C75A70F75F1FE75F2FF75F32E
:104509000775F47875A4BA75A5FF75A60775AE0089
:1045190075AFFF75D48175D5FF75D6FF75D7FF7552
:10452900A70075A20175A14775F80975D80075D955
:104539000475DA0975DB0975DC0975DD0975DE09AC
:1045490075D84075A71075D80075D90475DA09753D
:10455900DB0975DC0975DD0975DE0975D84075A7B4
:104569000075E60875E71075BC0175BE0475BD6C6C
:1045790075BE0775BDA075BE0875BD0175BC007512
:10458900BB1875BC2075BA0875E88075D11375A775
:104599000F75E10575E20075C7401242297597004C
:1045A900759780740A1267037597C0E59754207050
:1045B9000280F8758F0275A700D2AF75980075A9AA
:1045C9000C75A70F75AB4375ADFB75AC1E75A710C0
:1045D90075C91875CA0075CB0075C80475A700752B
:1045E9008912758E04758C00758A00C2A9D28C75E2
:1045F9008D00758B00D2ABD28E75EF0675D944C28A
:104609009974C8F5097508001200E975B500120416
:10461900E974639007B6F8E4F0E8A3F0120375743F
:10462900C89007B6F8E4F0E8A3F07464F5097508D2
:10463900001200E9900059E0900083F0900083E0B7
:10464900D39403400C7400900083F07400900059D7
:10465900F0C21D900083E0906085F82828738028B7
:10466900A2B44002D21D802075A70F75F30F75A75C
:1046790000A2A34002D21D800F75A70F75F317750D
:08468900A700A2A44002D21D0B
:0C6085000246670246690246710246822C
:10469100A21DB3405F757308E573D3940E5020E5F6
:1046A100739007B6F8E4F0E8A3F01202447464F5DD
:1046B100097508001200E97873740126F650D9745F
:1046C100029000BFF0900059E0900083F0900083C9
:1046D100E0906091F8282873801674009000E9F04A
:1046E100800E74009000CEF0800674009000DBF024
:0C6091000246D90246DB0246E30246EB61
:1046F100D21C805D757301E573D394075020E57377
:104701009007B6F8E4F0E8A3F01202447464F509E6
:104711007508001200E97873740126F650D9740106
:104721009000BFF0900059E0900083F0900083E08A
:1047310090609DF8282873801674009000E9F0803D
:0F4741000E74009000CEF0800674009000DBF044
:0C609D0002473802473A02474202474AD5
:10475000C21C900058E0900114F0900059E09000C5
:1047600083F090005AE09000A3F090005BE090008E
:10477000CCF090005CE0900078F090005DE090005C
:10478000BEF090005EE09000DCF090005FE09000F2
:10479000B0F0900060E09000CEF0900061E09000FA
:1047A000FEF0900062E0900162F0900063E0900102
:1047B00063F0900064E0900164F0900162E0700C9E
:1047C000900163E07006900164E060028004C227FB
:1047D0008002D2279000C9E07006740A9000C9F0E8
:1047E0009000AAE0700674E39000AAF09000B0E098
:1047F00004900071F09000B1E09000E3F0123BC42F
:10480000E5B54401F5B57406900047F074019000D9
:1048100048F0740390004AF0740590004BF0742D3A
:1048200090004CF0740590004DF0740190004EF033
:104830007400900053F07400900056F074FF9000E4
:1048400057F0745390014DF0747590014EF07462FE
:1048500090014FF07461900150F07472900151F02A
:104860007475900152F07420900153F074349001EB
:1048700054F07443900155F07479900156F0746CC3
:10488000900157F07420900158F07433900159F062
:10489000743690015AF0745490015BF09000E5E09A
:1048A00090006AF090009CE090006BF090009DE01A
:1048B00090006CF0A2B6B3920EA2B3B3920FA2A472
:1048C000B39223A2B4B39224A2A3B392259000661C
:1048D000E4F0756F00743A900776F074FD900777F6
:1048E000F0900067E4F09007B0E0FEA3E0FF7403EF
:1048F00012672374011200399007AEEEF0A3EFF0B7
:10490000756E01900045E4F0C222756300C213D2B7
:1049100014C202757100C22AD203C22BD204C22C67
:10492000D205C22DD206C22ED207C22FD208C23063
:10493000D209C231D20AC232D20BC233D20CC21E49
:10494000C21FC220C221C22612009E755F00756B75
:1049500000756100756532756600756700756800E1
:10496000756900756A00900015E4F0A3F0756C009D
:10497000D2B2D2A4D2B0D2B1D2A3D2A7D2A6D2A55B
:10498000D2B7900082E0D394FA400674FA90008285
:10499000F07E017F0090006CE012672390006BE0D6
:1049A0002FFF50010E90001FEEF0A3EFF0EFD39415
:1049B000FFEE940F400790001FE4F0A3F090006A10
:1049C000E0700674FF90006AF09000BFE0D394029C
:1049D000400674019000BFF09000C0E07005756D56
:1049E000028003756D039000C1E0D394014006740A
:1049F000009000C1F09000C7E0C3940A5006740A0A
:104A00009000C7F09000D1E0700674019000D1F0E2
:104A10009000D1E0B4FF0674FE9000D1F09000D871
:104A2000E0D394FE400674FE9000D8F09000FEE0C3
:104A3000D39402400674019000FEF0900114E0D37C
:104A4000940140067401900114F074019000DEF0AE
:104A500074019000DFF074009000E6F074009001A3
:104A600002F07400900106F074299006BCF0742ADC
:104A70009006C0F074179006C4F0741B9006D4F032
:104A8000741C9006D8F0D29C9000B1E0D3940440FE
:104A90000674049000B1F0E570D394104003757073
:104AA000109006BDE0D3940C400674009006BDF053
:104AB0009006C1E0D3940C400674009006C1F090BB
:104AC00006C5E0D3940C400674009006C5F090062D
:104AD000C9E0D3940C400674009006C9F09006CD4E
:104AE000E0D3940C400674009006CDF09006D1E01F
:104AF000D3940C400674009006D1F09006D5E0D314
:104B0000940C400674009006D5F09006D9E0D3943A
:104B10000C400674009006D9F09006DDE0D3940CAA
:104B2000400674009006DDF09006E1E0D3940C405E
:104B30000674009006E1F0D2EC75CF01A298B34064
:104B400005C298120646E54D6006A299B3B340022D
:104B50008005C299120C57E54E64016005E54EB41C
:104B6000040280D5C28E7E107F00E564126723E5C3
:104B70008D75F010A4FDACF0EF2DFDEE3CFCE58B47
:104B800075F01084FF7E00ED2FFFEC3EFE8E548FFB
:104B900055D28E9000A3E060099000A3E0C3943D3D
:104BA0004002805C900017126731900017E0FEA36E
:104BB000E0FF900019E0FCA3E0FDEFB50542EEB583
:104BC000043EB21BA20DB3401975E700A21BB3400F
:104BD00008E5B54404F5B58006E5B554FBF5B575B3
:104BE000E710900019E0FEA3E0FF90001BE0FCA39B
:104BF000E0FDEF2DFDEE3CFC900019ECF0A3EDF094
:104C00009000B0E060099000B0E0C39403400280DF
:104C10006F122D96A20DB35009900066E0C3942B3D
:104C20004002800690009AE0F545E54575F005A440
:104C3000FFAEF09007B8EEF0A3EFF0900087E0C36E
:104C400095614007E55FC3956050079007B8E4F0B1
:104C5000A3F0AE2EAF2F9007B8E0FCA3E0FDEFD39A
:104C60009DEE9C4004C2A1800B900066E0C394417D
:104C70005002D2A19000B0E0B40205A2A1B392A26A
:104C80009000B0E0B4031C122EB1AE2EAF2F9007EF
:104C9000B8E0FCA3E0FDEFD39DEE9C4004D2A180E0
:104CA00002C2A190008BE06009A2B3300F01B3B340
:104CB00040028039A2B3300F01B34031A2B33011AA
:104CC00001B3401C9000BEE0B40306A21EB3B34083
:104CD0000280067404900045F0D21EA211B3920F18
:104CE000A211B330B301B34004A211920FA2B630A7
:104CF0000E01B3500302537CA2B6300E01B3500331
:104D000002537CA2B6301001B350030251A1756E5C
:104D1000009000A3E0B43D1975E700A210B340086D
:104D2000E5B554FBF5B58006E5B54404F5B575E782
:104D300010055EA212B3B35013AE54AF55900008E5
:104D4000E0FCA3E0FDEDC39FEC9E4003024EA3E513
:104D50005EB41106755E13024E86E56DB4032EA295
:104D600028B34022E55EB42303756D01E55EC3946C
:104D70002350069000457401F0E55ED3942340066D
:104D80007402900045F0755E01D228805AE56DB43A
:104D90000206756D01755E23E55EB42305755E013F
:104DA0008045900045E07030E55EC3942350069046
:104DB00000457401F0E55ED3942340067402900030
:104DC00045F0E55EC394235002D222E55ED39423DE
:104DD0004002D222C296C2959000C0E0B4010512F2
:104DE00042298003755E019000A3E060099000A352
:104DF000E0C3943D40028043900017E0FEA3E0FF33
:104E00009000A3E08E048F05FF12671374018C06D7
:104E10008D0712003990001BEEF0A3EFF090001BFD
:104E2000E0F8A3E0900019C8F0A3C8F0900017E4E0
:104E3000F0A3F0C21BE5B554FBF5B5A2B4B3400234
:104E4000C224A2A4B34002C223A2A3B34002C2253B
:104E5000A222B34002C222A21EB34006A220921F89
:104E60008002B21F90008BE06012E56D700EA21EF2
:104E7000B35009A21F302001B3B34002800674056D
:104E8000900045F0C21EAE56AF57AC54AD55EF2D55
:104E9000FDEE3CFC74028C068D071200398E568F95
:104EA00057803AAE56AF57AC54AD55EF2DFDEE3CA2
:104EB000FC74018C068D071200398E568F57E56DF4
:104EC000C39402500DAC54AD557410C39D74279C0F
:104ED000400280091242297406900045F0E55EB454
:104EE0001403755E16E55EB423127403900045F05A
:104EF000D2229000C0E0B40103124229AE58AF594B
:104F0000AC54AD55EF2DFDEE3CFC8C588D59AE5494
:104F1000AF55EFD39DEE9C401190000FE0FAA3E057
:104F2000FBEBC394E8EA94034002800690000F1262
:104F3000673190000CE0FEA3E0FFAC54AD55EF2DBF
:104F4000FDEE3CFC90000CECF0A3EDF09000C0E016
:104F5000B40118AE54AF55740512672374011200E2
:104F600039900008EEF0A3EFF08011AE54AF557405
:104F700002126723900008EEF0A3EFF0C28E758D49
:104F800000758B00756400755501755400D28EE56F
:104F90005E240875F00984AFF07E00EF4E707590C6
:104FA000000CE0F8A3E090000AC8F0A3C8F090005D
:104FB0000AE0FEA3E0FFEF4E600B7C7B7D8912666A
:104FC000118E528F5390000CE4F0A3F0AE52AF5309
:104FD0007428BE00039F5010E5632FFF50010E742C
:104FE000011200398E528F538553639000C7E0A899
:104FF00052B8000DD395534008E553900044F0801B
:10500000099000C7E014900044F0E56D6006755308
:10501000007552009000BEE0B4030890003DE065CA
:105020005E6002800BA21FB34004D2218002B22135
:10503000E55E640B6005E55EB41D099000B0E060BC
:10504000031223D2900042E0655E6007900043E0C7
:10505000B55E03756F00A213B35006A212B3B3403E
:105060000302510990007CE0B401739000FEE0B4AB
:105070000214120E2690006FE075F0BEA4FFAEF091
:105080008E5C8F5D8056E56775F00A84FF7E009028
:10509000057612674AE0F55B755A00AE5AAF5B9031
:1050A00000A1E012672374648E048F05FF1267135A
:1050B0008C5C8D5DE55D90000EF0AE5AAF5B9000AC
:1050C0007AE012672374648E048F05FF12671374ED
:1050D000BE8C068D071267238E5C8F5D8017900053
:1050E0007AE075F0BEA4FFAEF08E5C8F5D9000A1FB
:1050F000E090000EF0E561C394CC5006E55D455CA0
:1051000070028003124325D213E56DB40106E55EFB
:10511000640B600280097570019000467401F0E52F
:105120006D70799000C3E0600D90006EE0A852B8F9
:1051300000069553400280389000C3E0B4021790F7
:10514000003BE0655E600790003CE0B55E03757073
:1051500003756C00800CC200756C00900015E4F0C3
:10516000A3F090006EE060067409900045F0802C7A
:1051700090003BE0655E600790003CE0B55E037523
:10518000700190003BE0B55E069000467401F0901F
:10519000003CE0B55E067402900046F0A210B392A7
:1051A0000EA210B330B601B3500302537C756E01EA
:1051B0009000A3E0B43D1975E700A210B34008E5E4
:1051C000B54404F5B58006E5B554FBF5B575E710B3
:1051D000E5B54401F5B5742B900066F0A210920E6F
:1051E000E55ED3944A4014D212E55ED3946D400B31
:1051F0007404900045F0D222755E469000CBE0B476
:105200000107E56AC394144002800912422974130D
:10521000900045F0A22A300301B3501D75E700A2AB
:105220002AB34008E5B54408F5B58006E5B554F75E
:10523000F5B575E710A22A9203A22B300401B350F2
:105240001D75E700A22BB34008E5B54402F5B58013
:1052500006E5B554FDF5B575E710A22B9204A22C16
:10526000300501B3500FA22CB34004D2A08002C27B
:10527000A0A22C9205A22D300601B3500FA22DB38F
:105280004004D2978002C297A22D9206A22E300728
:1052900001B3500FA22EB34004D2A28002C2A2A238
:1052A0002E9207A22F300801B3500FA22FB3400453
:1052B000D2A18002C2A1A22F9208A230300901B36C
:1052C000501D75E700A230B34008E5B54440F5B580
:1052D0008006E5B554BFF5B575E710A2309209A276
:1052E00031300A01B3501D75E700A231B34008E523
:1052F000B54480F5B58006E5B5547FF5B575E71082
:10530000A231920AA232300B01B3500FA232B34045
:1053100004D2878002C287A232920BA233300C01E2
:10532000B3500FA233B34004D2908002C290A23394
:10533000920CE56AC394415009740E900045F01236
:10534000422990004DE0FE900049E0C39E40099044
:105350000049E0D39408400974FB900045F01242E4
:1053600029900052E06015900052E0FE90004CE061
:105370006E600974FE900045F0124229A222B340EB
:1053800004C296C2959000FBE0600CAE52AF53741D
:1053900014BE00059F40028048900083E09060A901
:1053A000F8282873803BA2B4B35005A224B340026E
:1053B000800512437DD2248028A2A3B35005A225E4
:1053C000B34002800512437DD2258015A2A4B350BC
:1053D00005A223B34002800512437DD223800280C0
:0153E00000CC
:1060A9000253A40253A60253B90253CC0253DF028E
:0260B90053E1B1
:1053E100A215B3B3500890003DE0655E600302541E
:1053F100C0A201B35006A200B3B340030254BC9053
:1054010000BEE0B403028003025491A20DB34067D1
:10541100A221B3402D123A67E55DF5FBE55CF5FC91
:10542100D293A202B34002D2879000DCE0B4021012
:10543100123A94E55DF5FBE55CF5FC75A700D287B2
:105441008033123A67E55DF5EBE55CF5ECD291A2AC
:1054510002B34006E5B54410F5B59000DCE0B402B6
:1054610014123A94E55DF5EBE55CF5EC75A700E502
:10547100B54410F5B58017123A67E55DF5FBE55CBB
:10548100F5FCE55DF5EBE55CF5ECD293D291802B73
:10549100123A67E55DF5FBE55CF5FCD293A202B338
:1054A1004002D2879000DCE0B40210123A94E55D2C
:1054B100F5FBE55CF5FC75A700D287C215D216A2F3
:1054C10016B3B3500890003EE0655E600302559F3D
:1054D100A201B35006A200B3B3400302559B900052
:1054E100BEE0B403028003025570A20DB34067A26F
:1054F10021B3402D123A67E55DF5E9E55CF5EAD2A5
:1055010094A202B34002D2909000DCE0B4021012E7
:105511003A94E55DF5E9E55CF5EA75A700D290807E
:1055210033123A67E55DF5EDE55CF5EED292A20244
:10553100B34006E5B54420F5B59000DCE0B40214B3
:10554100123A94E55DF5EDE55CF5EE75A700E5B57C
:105551004420F5B58017123A67E55DF5E9E55CF59C
:10556100EAE55DF5EDE55CF5EED294D292802B1281
:105571003A67E55DF5E9E55CF5EAD294A202B3404C
:1055810002D2909000DCE0B40210123A94E55DF58D
:10559100E9E55CF5EA75A700D290D215C216E5706F
:0E55A1009060BBF82828730259F69000B1E024
:0660BB000255A80255ABDE
:1055AF009060EEF8282873121EAE8012121EAE8085
:0E55BF000D121F388008121FE48003121FE433
:0F60EE000255B60255BB0255C00255C50255CA30
:1055CD007570020259F6122110122227A238B3402B
:1055DD00229000A5E0F56C900076E0256CFE900021
:1055ED0044E075F01E84FC7F00EE2CF536741090AF
:1055FD000045F09007AEE0FEA3E0FF740A126723AA
:10560D0090000AE0FCA3E0FD74098F02FF126713FE
:10561D008D078C038E048A058B061266119007B2D6
:10562D00EEF0A3EFF074F0BE00039F500B74F090FA
:10563D0007B2F8E4F0E8A3F0E53670037536019093
:10564D0007B2E0FEA3E0FFE5362FFF50010E9007F5
:0D565D00B2EEF0A3EFF0757003900046E090
:0360C1000255D3B2
:10566A009060FDF82828738010A239400375700AEB
:09567A008007A239400375700B92
:0960FD0002567102567302567C32
:105683000259F69006BDE060031224EA9000FCE0A4
:10569300B401149000FDE0A852B8000495535007DC
:1056A300E55FC39560400280097415900045F002E0
:1056B30057369000B1E0D39402403F900085E02438
:1056C30003A852B8000495535009900087E0D3957E
:1056D3006150028008D2017408900045F090008563
:1056E300E0A852B80005D39553500B900087E024EF
:1056F30003C395615002C2018039900085E0240301
:10570300A852B8000495535007E55FC39560400263
:105713008008D2017408900045F0900085E0A852FB
:10572300B80005D395535009E560240FC3955F5026
:1057330002C2019000CBE07007E56AC394144002F3
:105743008002D201A2014005757004800A757010B1
:10575300900015E4F0A3F0A20DB34029E56775F0BE
:105763000A84FF7E0090057612674AE0C39469506D
:1057730005122407800F9007B0E0F8A3E09007AE6E
:0C578300C8F0A3C8F00259F69000B1E095
:0660C40002568602578B14
:10578F00906106F8282873120F108012120F1080E4
:0E579F000D1210BE80081211708003121170DE
:0F61060002579602579B0257A00257A50257AAAD
:1057AD009006C1E060031225C67570050259F61208
:1057BD0012B07570069006C5E060031226B690060D
:1057CD00C9E060031227920259F690000EE06006C0
:1057DD00A20DB3B34002801D90000EE02529FFAE4F
:1057ED002850010E8E288F29E55ED3941250069015
:1057FD00000EE014F01214F67570079006CDE060FF
:10580D000312286E9006D1E0600312294A0259F660
:10581D009000FEE0B40203120E9E1218F57570088A
:10582D009006D5E06003122A269006D9E060031297
:10583D002B020259F6121CB1A215B35005A216B3D4
:10584D0040028004D215D2167570109006DDE0600E
:10585D0003122BDE9006E1E06003122CBA0259F61A
:10586D000259F6900035E0C394465008C29674462E
:10587D00900035F090003FE0B4011DE536240AF5A7
:10588D00369007B2E0FEA3E0FF740A2FFF50010E21
:10589D009007B2EEF0A3EFF090003FE0B4021DE5EB
:1058AD00362414F5369007B2E0FEA3E0FF74142FF2
:1058BD00FF50010E9007B2EEF0A3EFF085365B7549
:1058CD005A0090003BE0F573123ADFE55D9000352C
:1058DD00F0900004E55AF0A3E55BF0E57390003617
:1058ED00F0C2189007B2E0F55AA3E0F55B90003BCB
:1058FD00E0F573123ADFE55D900033F0900000E5BE
:10590D005AF0A3E55BF0E573900034F0C217E56D36
:10591D00B4010575700B80037570030259F6900084
:10592D0039E0C3944650139000CCE0B40104C29604
:10593D008002C2957446900039F0900040E0B401A9
:10594D001DE536240AF5369007B2E0FEA3E0FF749C
:10595D000A2FFF50010E9007B2EEF0A3EFF090006A
:10596D0040E0B4021DE5362414F5369007B2E0FE92
:10597D00A3E0FF74142FFF50010E9007B2EEF0A3B9
:10598D00EFF085365B755A0090003CE0F573123AE6
:10599D00DFE55D900039F0900006E55AF0A3E55B78
:1059AD00F0E57390003AF0C21A9007B2E0F55AA3F1
:1059BD00E0F55B90003CE0F573123ADFE55D900099
:1059CD0037F0900002E55AF0A3E55BF0E573900027
:1059DD0038F0C219E56DB40103756D007570038063
:0959ED000880068004800280009D
:1060CA000257BC0257D702581D02584202586D02A5
:1060DA00587002592B0259EE0259F00259F202592C
:0460EA00F40259F66D
:1059F600900033E0B55E028003025A98A217407207
:105A0600900000E0FEA3E0FFEF4E6021AE56AF57D8
:105A1600900000E0FCA3E0FD120003740A8E048FE0
:105A260005FF126713900000ECF0A3EDF090003430
:105A3600E0601A900000E0FEA3E0FFAC56AD57EF21
:105A46002DFDEE3CFC900000ECF0A3EDF090003450
:105A5600E0D39401401A900000E0FEA3E0FFAC56AC
:105A6600AD57EF2DFDEE3CFC900000ECF0A3EDF001
:105A7600D217AE54AF55900000E0FCA3E0FDEFC393
:105A86009DEE9C400D1243CAD296C21774C8900070
:105A960033F0A217B3B35007900033E0B55E02802F
:105AA6000D1243CAD29674C8900033F0C217900004
:105AB60035E0B55E028003025B53A2184072900087
:105AC60004E0FEA3E0FFEF4E6021AE56AF57900014
:105AD60004E0FCA3E0FD120003740A8E048F05FFA8
:105AE600126713900004ECF0A3EDF0900036E0602E
:105AF6001A900004E0FEA3E0FFAC56AD57EF2DFD73
:105B0600EE3CFC900004ECF0A3EDF0900036E0D300
:105B16009401401A900004E0FEA3E0FFAC56AD5796
:105B2600EF2DFDEE3CFC900004ECF0A3EDF0D21856
:105B3600AE54AF55900004E0FCA3E0FDEFC39DEE2C
:105B46009C400AC2967446900035F0C218A218B35B
:105B5600B35007900035E0B55E02800AC2967446DF
:105B6600900035F0C218900037E0B55E028003025F
:105B76005C0EA2194072900002E0FEA3E0FFEF4E19
:105B86006021AE56AF57900002E0FCA3E0FD120084
:105B960003740A8E048F05FF126713900002ECF05F
:105BA600A3EDF0900038E0601A900002E0FEA3E05A
:105BB600FFAC56AD57EF2DFDEE3CFC900002ECF02D
:105BC600A3EDF0900038E0D39401401A900002E073
:105BD600FEA3E0FFAC56AD57EF2DFDEE3CFC90006A
:105BE60002ECF0A3EDF0D219AE54AF55900002E0EE
:105BF600FCA3E0FDEFC39DEE9C400D1243CAD29577
:105C0600C21974C8900037F0A219B3B350079000B8
:105C160037E0B55E02800D1243CAD29574C8900073
:105C260037F0C219900039E0B55E028003025CC904
:105C3600A21A4072900006E0FEA3E0FFEF4E60213C
:105C4600AE56AF57900006E0FCA3E0FD12000374C9
:105C56000A8E048F05FF126713900006ECF0A3ED81
:105C6600F090003AE0601A900006E0FEA3E0FFAC78
:105C760056AD57EF2DFDEE3CFC900006ECF0A3ED83
:105C8600F090003AE0D39401401A900006E0FEA39B
:105C9600E0FFAC56AD57EF2DFDEE3CFC900006EC58
:105CA600F0A3EDF0D21AAE54AF55900006E0FCA377
:105CB600E0FDEFC39DEE9C400AC295744690003904
:105CC600F0C21AA21AB3B35007900039E0B55E02CB
:105CD600800AC2957446900039F0C21A9000CEE050
:105CE600B402028003025DFE900068E0D395665020
:105CF60064900068E0F4042566FE9000D1E08E0012
:105D0600F5F0E884FF7E008F73EFC39410500CEF1C
:105D16008573F0A4FDACF08D7380037573FF90005E
:105D260068E0D39573400B900068E0C39573F571F6
:105D360080037571009000ECE0D3957140069000E9
:105D4600ECE0F5719000EDE0C3957150069000ED22
:105D5600E0F5718071900068E0C39566FE9000D111
:105D6600E08E00F5F0E884FF7E008F73EFC3941099
:105D7600500CEF8573F0A4FDACF08D738003757342
:105D8600FF85735B755A00900068E0255BFFAE5A8D
:105D960050010E8E5A8F5B74FFBE0009D39F4005DB
:105DA600855B7180037571FF9000ECE0D3957140BF
:105DB600069000ECE0F5719000EDE0C39571500699
:105DC6009000EDE0F571A20DB3B3500D900069E0BF
:105DD600FE9000D9E0D39E5002800A7407900045D9
:105DE600F0C2A2801375A710E5CDC395714004C219
:105DF600A28002D2A275A700E56FC39409500AA239
:105E0600EDB34005C2ED123050AE54AF557410C319
:105E16009F74279E400C900067E0C3945A4003028B
:105E26006082A212B340091242297406900045F01E
:105E3600A21DB34008E5B54404F5B58006E5B554A2
:105E4600FBF5B5A214B3500EE561D394334007E5D4
:105E560061C394CC400280419000FEE0B40214126B
:105E66000E2690006FE075F050A4FFAEF08E5C8FAA
:105E76005D800F90007AE075F050A4FFAEF08E5C66
:105E86008F5DE55D455C6011E5B54401F5B5742BA4
:105E9600900066F0124325D214900067E0D3940177
:105EA6004007E561C3941A40028002C2149006BD01
:105EB600E060031224EAA22A300301B35017A22A93
:105EC600B34008E5B54408F5B58006E5B554F7F5E1
:105ED600B5A22A92039006C1E060031225C6A22B42
:105EE600300401B35017A22BB34008E5B54402F5C0
:105EF600B58006E5B554FDF5B5A22B92049006C50E
:105F0600E060031226B6A22C300501B3500FA22C76
:105F1600B34004D2A08002C2A0A22C92059006C96A
:105F2600E06003122792A22D300601B3500FA22D76
:105F3600B34004D2978002C297A22D92069006CD56
:105F4600E0600312286EA22E300701B3500FA22E76
:105F5600B34004D2A28002C2A2A22E92079006D11A
:105F6600E0600312294AA22F300801B3500FA22F76
:105F7600B34004D2A18002C2A1A22F92089006D5F6
:105F8600E06003122A26A230300901B35017A2306E
:105F9600B34008E5B54440F5B58006E5B554BFF510
:105FA600B5A23092099006D9E06003122B02A23105
:105FB600300A01B35017A231B34008E5B54480F565
:105FC600B58006E5B5547FF5B5A231920A9006DD97
:105FD600E06003122BDEA232300B01B3500FA23267
:105FE600B34004D2878002C287A232920B9006E1A8
:105FF600E06003122CBAA233300C01B3500FA23367
:10600600B34004D2908002C290A233920C900067F3
:10601600E0C3945A5010E56FB40909900067E00494
:10602600F0756F00803BE56FB40903756F00755519
:1060360000755400758D00758B00756400900066C0
:10604600E0C394415008900066E004F08006744175
:10605600900066F0900066E0B44106E5B554FEF5A2
:10606600B5900067E0D394014007E56AC3944140C8
:0F607600028009740E900045F0124229024B3946
:106115000000010001400160018001A001C001E013
:1061250002000300039603B603D603F4040005003A
:106135000512052405360548055A056C057E0590AA
:1061450005A805C005DE0600061406280646066EE7
:1061550006AE05CF00FF013F015F017F019F01BF33
:1061650001DF01FF02FF039503B503D503F303FF29
:1061750004FF05110523053505470559056B057D03
:10618500058F05A705BF05CE05F1061306270645AC
:10619500066D06AD06ED05DD0FAA0FA50F9F0F9A3B
:1061A5000F940F8D0F870F800F780F710F680F6099
:1061B5000F570F4E0F450F3B0F300F250F1A0F0EC0
:1061C5000F020EF50EE80EDB0ECC0EBE0EAE0E9FC8
:1061D5000E8E0E7D0E6C0E5A0E470E340E200E0CD2
:1061E5000DF70DE20DCB0DB50D9D0D850D6D0D5406
:1061F5000D3A0D200D050CE90CCE0CB10C940C7666
:106205000C580C3A0C1B0BFB0BDB0BBB0B9A0B79DD
:106215000B570B350B130AF10ACE0AAB0A870A6432
:106225000A400A1C09F809D409B0098C0967094311
:10623500091F08FB08D608B2088E086A0846082315
:1062450007FF07DC07B9079607730751072F070DE7
:1062550006EC06CA06AA068906690649062A060A3A
:1062650005EC05CD05B0059205750558053C0520DD
:10627500050504EA04CF04B5049C048204690451AD
:1062850004390422040B03F403DE03C803B2039D9F
:10629500038903750361034D033B032803160304B8
:1062A50002F202E102D102C002B002A00291028212
:1062B5000273026502570249023C022F02220216AE
:1062C500020901FD01F201E601DB01D001C601BBB6
:1062D50001B101A7019D0194018B01820179017032
:1062E500016801600158015001480141013901323D
:1062F500012B0125011E01180111010B010500FFEC
:1063050000FA0FA60FA00F990F920F8B0F840F7C29
:106315000F740F6B0F620F580F4E0F430F380F2C72
:106325000F1F0F120F050EF70EE80ED80EC80EB789
:106335000EA50E930E800E6C0E580E420E2C0E15E9
:106345000DFD0DE40DCB0DB10D950D790D5D0D3FD9
:106355000D200D010CE10CC00C9E0C7C0C590C356C
:106365000C100BEA0BC40B9E0B760B4F0B260AFD8C
:106375000AD40AAA0A800A550A2A09FF09D409A8D3
:10638500097C0950092508F908CD08A10875084AAE
:10639500081E07F307C8079D07730749072006F777
:1063A50006CE06A6067E06570630060A05E405BF94
:1063B500059B057705540532051004EF04CE04AEA0
:1063C500048F047104530435041903FD03E203C764
:1063D50003AD0394037B0363034B0334031E0308DC
:1063E50002F302DE02CA02B602A30291027F026D27
:1063F500025C024C023C022C021D020E020001F25C
:1064050001E401D701CA01BE01B101A6019A018FBC
:106415000185017A01700166015D0153014A01415F
:10642500013901310129012101190112010B010471
:1064350000FD00F700F000EA00E400DE00D900D31B
:1064450000CE00C900C400BF00BA00B500B100AD60
:1064550000A800A400A0009C009900950091008E62
:0C646500008A008700840081007E007B1C
:10009E007547009007BAE4F0A3F075310075300093
:1000AE00754D00754E00C235D23674FE9007BCF801
:1000BE00E4F0E8A3F074FE9007BEF8E4F0E8A3F0D5
:1000CE0074FE9007C8F0745A9007C9F0745A9007DE
:1000DE00CAF0D237C229C239C23422750B00750A52
:1000EE0000AE0AAF0BAC08AD09EDC39FEC9E4016F7
:1000FE0074FF12670375CF01780B740126F6500456
:10010E0018E436F650DB22900041E0B4AA1C9007AA
:10011E0076E0B43C159007B6E0FEA3E0FFEF4E602C
:10012E0009741EBE0004D39F5003020243755D0086
:10013E00755C0075F8099007B6E0FEA3E0FF740742
:10014E006F4E6006740E6F4E7006743A900776F01E
:10015E009007B6E0FEA3E0FF7408BE001ED39F40DA
:10016E001A7E017F089007B6E0FCA3E0FD1DBDFFDF
:10017E00011C1200038E5A8F5B801F9007B6E0FEA3
:10018E00A3E0FF74081267678F048E057E017F0857
:10019E00CDCCCD1200038E5A8F5BAE5CAF5D740C6E
:1001AE00D39F74019E500302023EA2F9B3407EE536
:1001BE005D455C700375A382AE5CAF5D74016F4EDE
:1001CE00700375A300AE5CAF5D74026F4E700D9040
:1001DE0007B7E075F002A4FDACF08DA3AE5CAF5D89
:1001EE0074036F4E700375A300AE5CAF5D7403BEF7
:1001FE0000039F5013AC5AAD5BED2FFFEC3EFE900B
:10020E00007212674AE0F5A3AE5CAF5DEFB40B0966
:10021E00EEB401057414126703AE5CAF5DEFB40B60
:10022E0007EEB4010375F80D785C1267770201A82A
:10023E00900041E4F022755D00755C0075F8099040
:10024E0007B6E0FEA3E0FF7408BE001ED39F401A5F
:10025E007E017F089007B6E0FCA3E0FD1DBDFF0107
:10026E001C1200038E5A8F5B801F9007B6E0FEA310
:10027E00E0FF74081267678F048E057E017F08CD3C
:10028E00CCCD1200038E5A8F5BAE5CAF5D7411D372
:10029E009F74019E5003020374A2F9B3500302032C
:1002AE0071E55D455C700375A3D2AE5CAF5D740104
:1002BE006F4E700375A300AE5CAF5D74026F4E702F
:1002CE000D9007B7E075F002A4FDACF08DA3AE5C07
:1002DE00AF5D74036F4E700375A300AE5CAF5D74BB
:1002EE00046F4E700375A300AE5CAF5D74056F4E68
:1002FE00700375A300AE5CAF5D74066F4E70037530
:10030E00A300AE5CAF5D74076F4E700375A300AEB5
:10031E005CAF5D74086F4E700375A300AE5CAF5D8D
:10032E007408BE00039F5016AC5AAD5BED2FFFEC68
:10033E003EFE90006D12674AE5A3F075A300AE5C19
:10034E00AF5DEFB41009EEB401057414126703AE7D
:10035E005CAF5DEFB41007EEB4010375F80D785C79
:10036E0012677702029722755D00755C0075F809B9
:10037E00AE5CAF5D7417BE0004D39F500302044DF4
:10038E00A2F9B3500302044AE55D455C700375A300
:10039E00D2AE5CAF5D74016F4E700375A300AE5CA0
:1003AE00AF5D74026F4E700D9007B7E075F002A44A
:1003BE00FDACF08DA3AE5CAF5D74036F4E70037534
:1003CE00A300AE5CAF5D74046F4E700375A300AEF8
:1003DE005CAF5D74056F4E700375A300AE5CAF5DD0
:1003EE0074066F4E700375A300AE5CAF5D74076F3D
:1003FE004E700375A300AE5CAF5D74086F4E700354
:10040E0075A300AE5CAF5D7408BE00039F500C90E8
:10041E00004F12674AE5A3F075A300AE5CAF5D74A2
:10042E00166F4E70057414126703AE5CAF5D7416D2
:10043E006F4E700375F80D785C12677702037E229B
:10044E00900041E0B4AB0280030204E8755D0075D4
:10045E005C0075F809AE5CAF5D7412BE007CD39F74
:10046E004078A2F9B34070E55D455C700375A382D8
:10047E00AE5CAF5D74016F4E700375A300AE5CAFE2
:10048E005D74026F4E700D9007B7E075F002A4FD1B
:10049E00ACF08DA3AE5CAF5D74036F4E700375A3AD
:1004AE0000AE5CAF5D7403BE00039F500990005414
:1004BE0012674AE0F5A3AE5CAF5D74116F4E700526
:1004CE007414126703AE5CAF5D74116F4E700375DA
:1004DE00F80D785C126777020463229007C5E4F08A
:1004EE0074649007B6F8E4F0E8A3F012037574C8CC
:1004FE009007B6F8E4F0E8A3F074FF90004FF074A4
:10050E00FF900050F074FF900051F074009000497D
:10051E00F074FF900052F07400900054F07401904B
:10052E000055F090005BE0B4371A900058E0900050
:10053E004FF0900059E0900050F090005AE090007B
:10054E0051F080469007C57401F074659007B6F8B7
:10055E00E4F0E8A3F012037574C89007B6F8E4F05F
:10056E00E8A3F090005BE0B4371A900058E09000DA
:10057E004FF0900059E0900050F090005AE090003B
:10058E0051F0800674029007C5F09007C6E4F0742F
:10059E00669007B6F8E4F0E8A3F012037574C890FD
:1005AE0007B6F8E4F0E8A3F090005AE0B4371290E2
:1005BE000058E0900049F0900059E0900052F08011
:1005CE00769007C67401F074679007B6F8E4F0E809
:1005DE00A3F012037574C89007B6F8E4F0E8A3F020
:1005EE0090005AE0B43712900058E0900049F09015
:1005FE000059E0900052F0803E74029007C6F074ED
:10060E00689007B6F8E4F0E8A3F012037574C8908A
:10061E0007B6F8E4F0E8A3F090005AE0B437129071
:10062E000058E0900049F0900059E0900052F080A0
:10063E000674039007C6F022E54E64046006E59941
:10064E0064FF60028031A2354004D2358027E54E2A
:10065E00600874E6254E900045F0E54D600874F094
:10066E00254D900045F0E54EB4010280FE754E001A
:10067E00754D00C2358002C235E54E90384AF828D5
:10068E002873754E00E599B4FF03754D01E599B4D5
:10069E00FE03754D02E599B4FD03754D03E599B45E
:1006AE00FC03754D04E599B4FA03754D05E599B44F
:1006BE00FB06754E01124229E599B4F906754E04F2
:1006CE00124229E599D394E54007E599C394F04089
:1006DE0002801685994F754E027E017F00E54FC34D
:1006EE0094E61267238E328F339007BAE4F0A3F0AC
:1006FE00E599D394C44007E599C394E64002802857
:10070E0085994F754E0374E5C3954FF533753200D9
:10071E00AE32AF339061151266F2E493F874019322
:10072E009007BAC8F0A3C8F0D299020C56900058A0
:10073E00E07005A227B3400280429007BAE0FEA304
:10074E00E0FF74FFBE00039F5009EFC39446EE9482
:10075E000640119007BAE0FEA3E0FFEFD3946DEED2
:10076E00940640139007BAE0FEA3E0FF90007612C5
:10077E00674AE599F0800385997480119007BAE075
:10078E00FEA3E0FF90007612674AE599F09007BA53
:10079E001267319007BAE0FEA3E0FFEFB40106EE58
:1007AE00B4070280030209FD900776E0B43C028094
:1007BE00030209FDA22750030208E8C29C900058CC
:1007CE00E0900114F0900059E0900083F090005AF0
:1007DE00E09000A3F090005BE09000CCF090005C05
:1007EE00E0900078F090005DE09000BEF090005E2A
:1007FE00E09000DCF090005FE09000B0F0900060C0
:10080E00E09000CEF0900061E09000FEF09000626B
:10081E00E0900162F0900063E0900163F09000645C
:10082E00E0900164F0123BC490006AE09000E5F0A5
:10083E0090006BE090009CF090006CE090009DF0BA
:10084E0074639007B6F8E4F0E8A3F074AB9000413F
:10085E00F012044E900041E4F07464F5097508003E
:10086E001200E9A21C4039757301E573D394075049
:10087E002DE5739007B6F8E4F0E8A3F074AA9000A3
:10088E0041F0120115E573C39407500A7464F5091B
:10089E007508001200E97873740126F650CC803783
:1008AE00757308E573D3940E502DE5739007B6F863
:1008BE00E4F0E8A3F074AA900041F0120115E5737C
:1008CE00C3940E500A7464F5097508001200E97895
:1008DE0073740126F650CC0209E7C29C900114E015
:1008EE00900058F0900083E0900059F09000A3E043
:1008FE0090005AF09000CCE090005BF0900078E011
:10090E0090005CF09000BEE090005DF09000DCE0A6
:10091E0090005EF09000B0E090005FF09000CEE0AE
:10092E00900060F09000FEE0900061F07400900086
:10093E0062F07400900063F07400900064F07463D1
:10094E009007B6F8E4F0E8A3F074AB900041F01213
:10095E00044E900041E4F07464F50975080012002D
:10096E00E9757301E573D394075026E5739007B6C6
:10097E00F8E4F0E8A3F074AA900041F012011574A7
:10098E0064F5097508001200E97873740126F650B3
:10099E00D3D29C7599FB743C900776F0757308E57D
:1009AE0073D3940E5026E5739007B6F8E4F0E8A3DF
:1009BE00F074AA900041F01201157464F5097508DF
:1009CE00001200E97873740126F650D374C89007AC
:1009DE00B6F8E4F0E8A3F080FE74C89007B6F8E429
:1009EE00F0E8A3F0D29C754E00754D007599FB0290
:1009FE000C569007BAE0FEA3E0FFEF4E7006859905
:100A0E00317530009007BAE0FEA3E0FF74016F4E1F
:100A1E00701BAC30AD31AA32AB33ED2BFBEC3AFA96
:100A2E008A068B0790007612674AE599F09007BA0E
:100A3E001267319007BAE0FEA3E0FF74026F4E70AA
:100A4E0021AC30AD3174566D4C7006E54F64E660E6
:100A5E00028003124229123BC4854F99754E0075D0
:100A6E004D00020C569007BAE0FEA3E0FF90007610
:100A7E0012674AE599F09007BA1267319007BAE00B
:100A8E00FEA3E0FFAC32AD338F028E038C068D07D2
:100A9E009061591266F2E493F9740193FEEAD39EC3
:100AAE00EB994009854F99754E00754D00020C5615
:100ABE009007BAE0FEA3E0FF90007612674AE59930
:100ACE00F09007BA1267319007BAE0FEA3E0FFEF8D
:100ADE00B40006EEB401028003020C56900051E001
:100AEE00D394C7400B900051E0C394C8F550801AC0
:100AFE00900051E0D39463400B900051E0C3946496
:100B0E00F5508006900051E0F550E55075F002A4C6
:100B1E00FFAEF08F73EF900076126755EFFCE0FD9D
:100B2E00EC900079126755EDFCE0FDEC2DB550020E
:100B3E008003020C470FEF900076126755E573FFA6
:100B4E00E0FCEF90007A126755ECFFE0FCEFC39CDF
:100B5E00B550028003020C47E5739000781267557A
:100B6E00E573FFE0FCEF90007B126755ECFFE0FCB5
:100B7E00EF2CB550028003020C47E57390007C12F7
:100B8E006755E0C39550900058F0E57390007D12C4
:100B9E006755E0C39550900059F0E57390007E12B2
:100BAE006755E0C3955090005AF0740090005BF0CA
:100BBE0074FF90005CF0E573900080126755E0C3FF
:100BCE00955090005DF0E573900081126755E0C37B
:100BDE00955090005EF0E573900082126755E0C369
:100BEE00955090005FF0E57390007F126755E0C35B
:100BFE0095509007B6F8E4F0E8A3F074AB9000417E
:100C0E00F012044E7464F5097508001200E990079D
:100C1E00B612673112044E7464F50975080012009D
:100C2E00E99007B612673112044E7599F97464F59E
:100C3E00097508001200E980FE7599FF7464F509C4
:080C4E007508001200E980FEA8
:0F384A0002069002073B020A00020A73020ABE3E
:100C560022E54D903859F8282873020D699007BA95
:100C6600E0FEA3E0FF90004712674AE0F59990077F
:100C7600BA1267319007BAE0FEA3E0FF74116F4E17
:100C86007003754D00020D69856E99020D69900716
:100C9600BAE0FEA3E0FF90007612674AE0F599EF0E
:100CA600B40107EEB40703754D009007BA12673119
:070CB600020D699007BBE08D
:0F385900020C60020C63020C8E020C94020CB97C
:100CBD00903A0CF8282873855399020D5E855F993B
:100CCD00020D5E856199020D5E856599020D5E8549
:100CDD006799807D85689980788569998073856A23
:100CED0099806E900016E0F5998066A236B34007A4
:100CFD007599FAC2368041A226B3400575990F80C9
:100D0D00359007C5E0600A9007C5E024DCF59980B1
:100D1D00169007C6E0600A9007C6E024DEF59980BC
:100D2D0006900045E0F599900045E4F09007C5E484
:100D3D00F09007C6E4F0C2268017856B9980128566
:100D4D006699800D856C9980087599FC8003754DA9
:010D5D000095
:103A0C00020CC4020CCA020CD0020CD6020CDC0252
:103A1C000CE1020CE6020CEB020CF0020CF8020DAD
:0D3A2C0047020D4C020D51020D56020D5BBC
:0B0D5E009007BA1267318003123A3987
:03386800020D66E8
:100D690022E537255BFFAE5A50010E9000761267D7
:100D79004AE0F538E537255BFFAE5A50010E0FBF43
:100D890000010E90007612674AE0F539853F3BE590
:100D990038B539058538378041E539D39538401D4F
:100DA900E539C39538853AF0A4FFAEF0E53B8E04EA
:100DB9008F05FF126713ED2538F537801DE538C318
:100DC9009539853AF0A4FFAEF0E53B8E048F05FF17
:100DD900126713EDF4042538F53722E539D3953830
:100DE900401DE539C39538853AF0A4FFAEF0E53BDF
:100DF9008E048F05FF126713ED2538F537801DE541
:100E090038C39539853AF0A4FFAEF0E53B8E048FDF
:100E190005FF126713EDF4042538F5372290007C9D
:100E2900E0B40170E56775F00A84FF7E008F37E54D
:100E39006775F00A84ADF07C008D3A753F0A755AE2
:100E490005755B24E537C394115005120D6A8006B8
:100E59009005ABE0F537E53790006FF0E56775F081
:100E69000A84FF7E008F37E56775F00A84ADF07C50
:100E7900008D3A753F0A755A05755B5AE537C39473
:100E8900115005120D6A80069005E1E0F537E53746
:100E990090000EF02290007CE0B4016AE56775F0DD
:100EA9000A84FF7E008F37E56775F00A84ADF07C10
:100EB900008D3A753F0A755A05755B36E537C39457
:100EC900115005120D6A80069005BDE0F53785378A
:100ED9004BE56775F00A84FF7E008F37E56775F08B
:100EE9000A84ADF07C008D3A753F0A755A05755B29
:100EF90048E537C394115005120D6A80069005CF55
:100F0900E0F53785374C22E55F75F00484FF7E00F4
:100F19008F37E55F75F00484ADF07C008D3A753F3D
:100F290004755A01755B00E537C3943F5005120DEE
:100F39006A80069001B5E0F5378537297528009054
:100F49000044E075F020A4FFAEF09000C7E08E04E5
:100F59008F05FF1267138D379000AFE0D3955F506F
:100F6900030210169000D3E0D3955F4010ED900175
:100F7900B6126755E0F52B752A0002101390009EF2
:100F8900E0D3955F4043E5379001B6126755E0F528
:100F990038E5379001D6126755E0F5399000D3E06E
:100FA900F404255FF53A90009EE0FE9000D3E0F44A
:100FB900042EF53BE538B539058538378003120D20
:100FC900E485372B752A008041E5379001D61267F1
:100FD90055E0F538E5379001F6126755E0F5399097
:100FE900009EE0F404255FF53A9000AFE0FE900022
:100FF9009EE0F4042EF53BE538B539058538378090
:1010090003120DE485372B752A000210BD9000D616
:10101900E0D3955F5011E537900236126755E0F538
:101029002B752A000210BD90009FE0D3955F5043B5
:10103900E537900216126755E0F538E53790023624
:10104900126755E0F53990009FE0F404255FF53A01
:101059009000D6E0FE90009FE0F4042EF53BE538C1
:10106900B539058538378003120DE485372B752A84
:10107900008041E5379001F6126755E0F538E5370C
:10108900900216126755E0F5399000AFE0F4042597
:101099005FF53A90009FE0FE9000AFE0F4042EF572
:1010A9003BE538B539058538378003120DE48537B6
:1010B9002B752A00229000E7E0F53C753F11755A1F
:1010C90002755B00AE52AF53E53C75F00FA4FDAC61
:1010D900F0EDD39FEC9E4021E53C8E048F05FF1275
:1010E9006713ED75F010A4FFAEF0E55F75F011849C
:1010F900FD7C00ED2FF53D800EE55F75F01184FF55
:101109007E00EF24F0F53D853D37E55F75F01184EC
:10111900AFF07E008F3A120D6A85373EAE52AF535B
:101129009000E7E075F00FA4FDACF0EDD39FEC9EC5
:101139004028755A02755B10853D37120D6A853E48
:1011490038853739AE52AF53E53C8E048F05FF120F
:10115900673E8D3A853C3B120DE485372975280099
:10116900752B64752A00229000E7E0F53C753F1164
:10117900755A02755B00AE52AF53E53C75F00FA48A
:10118900FDACF0EDD39FEC9E4021E53C8E048F052C
:10119900FF126713ED75F010A4FFAEF0E56175F06D
:1011A9001184FD7C00ED2FF53D800EE56175F01190
:1011B90084FF7E00EF24F0F53D853D37E56175F04C
:1011C9001184AFF07E008F3A120D6A85373EAE5218
:1011D900AF539000E7E075F00FA4FDACF0EDD39F9D
:1011E900EC9E4028755A02755B10853D37120D6AD1
:1011F900853E38853739AE52AF53E53C8E048F05AD
:10120900FF12673E8D3A853C3B120DE485372975FF
:101219002800E56B6017E56BC394FE50109000DB66
:10122900E0B402099000C9E0D3940B50028017AED4
:1012390028AF29E56B12672374E78E048F05FF1227
:1012490067138C288D299000B1E0B40453E55F75CC
:10125900F00484FF7E008F37E55F75F00484ADF0FC
:101269007C008D3A753F04755A01755B00E537C3FB
:10127900943F5005120D6A80069001B5E0F537AE2E
:1012890028AF29E53712672374648E048F05FF128E
:101299006713AE28AF29EF2DFDEE3CFC8C288D2974
:1012A900752B64752A002290007CE0B40146E5673D
:1012B90075F00A84FF7E008F37E56775F00A84AD03
:1012C900F07C008D3A753F0A755A05755B00E53764
:1012D900C394115005120D6A8006900587E0F53711
:1012E900AE2AAF2BE5372FFF50010E7464126767E2
:1012F9008E2A8F2B90007DE0B40146E56875F00ACF
:1013090084FF7E008F37E56875F00A84ADF07C00B4
:101319008D3A753F0A755A05755B6CE537C39411AB
:101329005005120D6A80069005F3E0F537AE2AAF35
:101339002BE5372FFF50010E74641267678E2A8FD1
:101349002B90008CE0B40249E56AC3944175F0051D
:1013590084FF7E008F37E56A75F00584ADF07C0067
:101369008D3A753F05755A06755B00E537C39413C9
:101379005005120D6A8006900689E0F537AE2AAF4E
:101389002BE5372FFF50010E74641267678E2A8F81
:101399002B9000CEE0B40202800302144FE55F7582
:1013A900F01584FF7E008F37E55F75F01584ADF089
:1013B9007C008D3A753F15755A03755BF4E537C3A3
:1013C900940B5005120D6A8006900475E0F537E517
:1013D9003775F0FFA4FFAEF09000CFE08E048F05C3
:1013E900FF126713ED900068F0E56675F078A4FFC9
:1013F900AEF074FF8E048F05FF1267138C5A8D5B54
:1014090074028C068D071200398F37AC5AAD5B74A4
:1014190004FF12673E8D3A753F04755A06755B28BD
:10142900E537C3941D5005120D6A80069006BBE08E
:10143900F537AE2AAF2BE5372FFF50010E74641232
:1014490067678E2A8F2B90007BE0B4025DE561759A
:10145900F064A4FFAEF074081200398E5C8F5D74DD
:10146900058E048F05FF1267138D37AE5CAF5D746F
:10147900058E048F05FF12673E8D3A753F05755A33
:1014890005755BDEE537C394135005120D6A8006B6
:10149900900667E0F537AE2AAF2BE5372FFF5001ED
:1014A9000E74641267678E2A8F2B9000BDE0703C22
:1014B900900044E075F00584FF7E008F379000446A
:1014C900E075F00584ADF07C008D3A753F05755ADD
:1014D90005755BC0E537C3941D5005120D6A80067A
:1014E900900653E0F537E537900070F022900084BC
:1014F900E0B401179007C1E0252BFFAE2A50010E79
:101509009000D8E01267678E2A8F2B9000FCE0B418
:1015190001149000FDE0A852B8000495535007E566
:101529005FC39560400280129000A6E0252BFFAEB4
:101539002A50010E8E2A8F2B802F900084E0B4034D
:1015490016A229B3B350109007C4E0C39405A8525A
:10155900B800069553400280109000A6E0252BFFA5
:10156900AE2A50010E8E2A8F2B90007EE0B4020223
:1015790080030218F4900081E0602FE567D3944658
:10158900402890000FE0FEA3E0FF9000BCE075F05A
:1015990003A4FDACF0EFD39DEE9C400E9000E0E07B
:1015A900A852B80005D3955350030218F49000B11E
:1015B900E0B40302800302175885615B755A0090F5
:1015C9000088E0A852B800049553500E900089E0B5
:1015D900A85AB80005D3955B5003021755E5617504
:1015E900F002A4FFAEF074158E048F05FF12671385
:1015F9008C068D0790060612674AFEE0FFEE900002
:1016090080E0FEEF8E0088F0A4FFAEF074648E04D3
:101619008F05FF1267138C5A8D5B900044E075F0BB
:1016290018A4FFAEF09000C7E08E048F05FF126783
:10163900138C068D0790061E12674AAE5AAF5BE0FF
:1016490012672374648E048F05FF1267138C5A8DF9
:101659005BE565A85AB80077D3955B4072E565C329
:10166900955BFFE4955AFE8E5A8F5B7428BE000382
:101679009F500C755B28755A00740D900045F0AEAB
:101689005AAF5B900081E012672374288E048F059E
:10169900FF1267138C5A8D5BAE28AF29740A8E042A
:1016A9008F05FF1267138D068C07AC5AAD5BCFCE41
:1016B900CF120003740A8E048F05FF1267138C5A28
:1016C9008D5BAE28AF2912676F8E288F29807DE543
:1016D90065A85AB80004955B5072AE5AAF5BE565D0
:1016E9001267678E5A8F5B7428BE00039F500C7572
:1016F9005B28755A00740D900045F0AE5AAF5B90A7
:101709000081E012672374288E048F05FF12671386
:101719008C5A8D5BAE28AF29740A8E048F05FF128F
:1017290067138D068C07AC5AAD5BCFCECF12000381
:10173900740A8E048F05FF1267138C5A8D5BAE28CD
:10174900AF29EF2DFDEE3CFC8C288D290218F49071
:1017590000C9E0855FF0A4FFAEF074051267237439
:10176900071200398E5A8F5B900088E0A852B800A2
:101779000495535012900089E075F002A4FDACF075
:10178900EFC39DEE9C40030218F4E55F75F00B84EE
:10179900FF7E0090060612674AFEE0FFEE90008089
:1017A900E0FEEF8E0088F0A4FFAEF074648E048F23
:1017B90005FF1267138C5A8D5B900044E075F01891
:1017C900A4FFAEF09000C7E08E048F05FF126713E7
:1017D9008C068D0790061E12674AAE5AAF5BE0125F
:1017E900672374648E048F05FF1267138C5A8D5B0F
:1017F900E565A85AB80077D3955B4072E565C3954E
:101809005BFFE4955AFE8E5A8F5B7428BE00039FD6
:10181900500C755B28755A00740D900045F0AE5A4E
:10182900AF5B900081E012672374288E048F05FF57
:101839001267138C5A8D5BAE28AF29740A8E048FF8
:1018490005FF1267138D068C07AC5AAD5BCFCECF5F
:10185900120003740A8E048F05FF1267138C5A8DC8
:101869005BAE28AF2912676F8E288F29807DE565C9
:10187900A85AB80004955B5072AE5AAF5BE5651281
:1018890067678E5A8F5B7428BE00039F500C755B87
:1018990028755A00740D900045F0AE5AAF5B900060
:1018A90081E012672374288E048F05FF1267138C59
:1018B9005A8D5BAE28AF29740A8E048F05FF126713
:1018C900138D068C07AC5AAD5BCFCECF12000374D3
:1018D9000A8E048F05FF1267138C5A8D5BAE28AFF1
:1018E90029EF2DFDEE3CFC8C288D29229000DCE0AF
:1018F900B4026AE55F75F00884FF7E008F37E55F03
:1019090075F00884ADF07C008D3A753F08755A0171
:10191900755BE0E537C3943F5005120D6A80069068
:101929000275E0F53785372D752C00AE2CAF2DAC3F
:101939002AAD2B12000374648E048F05FF126713FE
:101949008C2C8D2D900079E08C068D0712672374FD
:10195900648E048F05FF1267138C2C8D2DAE28AF72
:1019690029AC2AAD2B12000374648E048F05FF1273
:1019790067138C288D29900079E08C068D071267F2
:101989002374648E048F05FF1267138C288D29A296
:101999000D401DAE52AF537405BE00039F5002D2D5
:1019A9000DE561D394CC4008D2017411900045F043
:1019B9009000DBE0B402089000C9E0640B6002808B
:1019C90035AE28AF29E56B12672374E78E048F05BE
:1019D900FF1267138C288D299000DCE0B40217AE42
:1019E9002CAF2DE56B12672374E78E048F05FF1268
:1019F90067138C2C8D2D90009BE05402601B900086
:101A090092E0A852B80012D39553400DA20DB3B37A
:101A19005007E561C3949A40028028AE34AF3590EF
:101A29000090E075F002A4FDACF0EF2DFDEE3CFC5A
:101A390074022DFD50010CE561BC0007D39D4003E4
:101A4900754301856135753400E5437003021B3820
:101A59009000EEE0C395435003021B2A9000FEE07C
:101A6900C394025076E56775F00A84FF7E009005FD
:101A79007612674AE0F55B755A00AE5AAF5B900083
:101A890091E012672374648E048F05FF1267138C2B
:101A99005C8D5D9000EEE004C395438C068D0712C2
:101AA90067239000EEE08E048F05FF1267138C5CAC
:101AB9008D5DAE28AF29EF2DFDEE3CFC8C288D29DC
:101AC9009000DCE0B40212AE2CAF2DAA5CAB5DEF46
:101AD9002BFBEE3AFA8A2C8B2D80469000EEE0041F
:101AE900C39543854BF0A4FFAEF09000EEE08E0461
:101AF9008F05FF1267138C5C8D5DAE28AF29EF2D22
:101B0900FDEE3CFC8C288D299000DCE0B40212AE7D
:101B19002CAF2DAA5CAB5DEF2BFBEE3AFA8A2C8B2E
:101B29002D05439000EEE0C39543500375430090A3
:101B3900009BE05401601B90008FE0A852B800128E
:101B4900D39553400DA20DB3B35007E55FC394CCB1
:101B59004002802590008DE075F003A4FFAEF0E50A
:101B6900402FFF50010E74032FFF50010EE55FBE99
:101B79000007D39F4003754401855F40E544700326
:101B8900021C6B9000EFE0C395445003021C5D906A
:101B990000FEE0C394025076E56775F00A84FF7E83
:101BA9000090057612674AE0F55B755A00AE5AAFA8
:101BB9005B90008EE012672374648E048F05FF1218
:101BC90067138C5C8D5D9000EFE004C395448C062F
:101BD9008D071267239000EFE08E048F05FF1267CF
:101BE900138C5C8D5DAE28AF29EF2DFDEE3CFC8C8E
:101BF900288D299000DCE0B40212AE2CAF2DAA5C2E
:101C0900AB5DEF2BFBEE3AFA8A2C8B2D80469000C8
:101C1900EFE004C39544854CF0A4FFAEF09000EFCB
:101C2900E08E048F05FF1267138C5C8D5DAE28AFC3
:101C390029EF2DFDEE3CFC8C288D299000DCE0B4C9
:101C49000212AE2CAF2DAA5CAB5DEF2BFBEE3AFA7C
:101C59008A2C8B2D05449000EFE0C3954450037501
:101C690044009000F1E02529FFAE2850010E8E288E
:101C79008F299000A0E0A828B80004952950099060
:101C890000A0E0F5297528009000DCE0B4020D9071
:101C990000A0E0A82CB80006952D4002800990000C
:101CA900A0E0F52D752C00229000DCE0B401028043
:101CB90003021DBCA20DB35003021DBA9000A7E098
:101CC900B40168AE28AF29AC52AD53120003743C7D
:101CD9008E048F05FF1267139000B7E0BC00109DBA
:101CE900400D9000B9E0A828B8000495295002D207
:101CF90002AE28AF29AC52AD53120003743C8E04D6
:101D09008F05FF1267139000B7E0C3940ABC001552
:101D1900D39D40119000B9E0C39405A828B80005E7
:101D2900D3952950028002C2028068AE28AF29AC3F
:101D390052AD5312000374788E048F05FF12671396
:101D49009000B7E0BC00109D400D9000B9E0A828B4
:101D5900B8000495295004D2028038AE28AF29ACC6
:101D690052AD5312000374788E048F05FF12671366
:101D79009000B7E0C3940ABC0015D39D40119000B0
:101D8900B9E0C39405A828B80005D3952950028065
:101D990002C202A202B34019AE28AF299000B8E0EE
:101DA90012672374648E048F05FF1267138C288DC4
:101DB900298002C202A200B34006A201B3B35009AE
:101DC900900015E4F0A3F08024AE28AF297400D365
:101DD9009F74019E400C900015E528F0A3E529F0B9
:101DE900800B74FF900015F8E4F0E8A3F09000BEB2
:101DF900E0D39402400C9000A9E07006A20DB3B3A1
:101E09004002801AAE28AF2974021267238E288FE8
:101E190029AE2CAF2D74021267238E2C8F2D9000C2
:101E2900A7E0B4011AAE28AF2974021267238E28DD
:101E39008F29AE2CAF2D74021267238E2C8F2DAEF5
:101E490028AF29745E126723740A8E048F05FF1266
:101E590067138C288D299000DCE0B40217AE2CAFF3
:101E69002D745E126723740A8E048F05FF1267139F
:101E79008C2C8D2DAE28AF297402BE000AD39F4049
:101E890006752902752800AE2CAF2D7402BE000A12
:101E9900D39F4006752D02752C00900013E528F09C
:101EA900A3E529F022900044E0900376126755E0FB
:101EB900F541754264900044E0FE9000B2E0D39E83
:101EC9004037E55F75F00884FF7E008F37E55F7561
:101ED900F00884ADF07C008D3A753F08755A03759A
:101EE9005B96E537C3941F5005120D6A800690046E
:101EF9002BE0F5378537428035E55F75F00884FFBB
:101F09007E008F37E55F75F00884ADF07C008D3A6F
:101F1900753F08755A03755BB6E537C3941F5005BD
:101F2900120D6A800690044BE0F5378537422290FE
:101F390000E8E0F53C753F11755A04755B00AE5237
:101F4900AF53E53C75F00FA4FDACF0EDD39FEC9ECB
:101F59004021E53C8E048F05FF126713ED75F010E3
:101F6900A4FFAEF0E55F75F01184FD7C00ED2FF55F
:101F79003D800EE55F75F01184FF7E00EF24F0F5DA
:101F89003D853D37E55F75F01184AFF07E008F3AEE
:101F9900120D6A85373EAE52AF539000E8E075F0F6
:101FA9000FA4FDACF0EDD39FEC9E4028755A047543
:101FB9005B10853D37120D6A853E38853739AE523B
:101FC900AF53E53C8E048F05FF12673E8D3A853C81
:101FD9003B120DE4853741754264229000E8E0F533
:101FE9003C753F11755A04755B00AE52AF53E53C21
:101FF90075F00FA4FDACF0EDD39FEC9E4021E53CBC
:102009008E048F05FF126713ED75F010A4FFAEF073
:10201900E56175F01184FD7C00ED2FF53D800EE53D
:102029006175F01184FF7E00EF24F0F53D853D37A1
:10203900E56175F01184AFF07E008F3A120D6A8563
:10204900373EAE52AF539000E8E075F00FA4FDACF7
:10205900F0EDD39FEC9E4028755A04755B10853DC1
:1020690037120D6A853E38853739AE52AF53E53C94
:102079008E048F05FF12673E8D3A853C3B120DE4B5
:102089008537417542649000B1E0B4047990004409
:10209900E0FE9000B2E0D39E4037E55F75F008841A
:1020A900FF7E008F37E55F75F00884ADF07C008D09
:1020B9003A753F08755A03755B96E537C3941F5007
:1020C90005120D6A800690042BE0F53785374280AA
:1020D90035E55F75F00884FF7E008F37E55F75F0A1
:1020E9000884ADF07C008D3A753F08755A03755B1D
:1020F900B6E537C3941F5005120D6A800690044B4C
:10210900E0F5378537422290007CE0B4013BE56772
:1021190075F00A84FF7E008F37E56775F00A84AD94
:10212900F07C008D3A753F0A755A05755B12E537E3
:10213900C394115005120D6A8006900599E0F53790
:10214900E5422537C39464F54290007DE0B4013B34
:10215900E56875F00A84FF7E008F37E56875F00A37
:1021690084ADF07C008D3A753F0A755A05755B7E22
:10217900E537C394115005120D6A8006900605E0F3
:10218900F537E5422537C39464F542E5412542F523
:1021990036900084E0B402109007C0E02536FE9026
:1021A90000D8E0F4042EF5369000DBE0D39401402A
:1021B90040E56BC394E7501D74E7C3956BFE900728
:1021C900C2E08E00F5F0E884FF7E008F37E5362502
:1021D90037F536801CE56BC394E7FE9007C2E08EA5
:1021E90000F5F0E884FF7E008F37E536C39537F5B3
:1021F90036A20D4006E5412464F536E536D39464EC
:102209004009E536C39464F53680037536009000BD
:10221900B4E0C3953650069000B4E0F53622D200FA
:1022290090006EE0A852B800049553504190006E9A
:10223900E0A852B800049553500375360F90006E0C
:10224900E004A852B800049553500375360A90006B
:102259006EE02402A852B80004955350057536055E
:10226900C20090006EE060067409900045F0C23922
:102279007E017F009000BAE01267239000C9E08ECA
:10228900048F05FF126713E55FBC0017D39D401348
:102299009000C3E0B40204D2398002C200740A90EB
:1022A9000045F09000BBE0C3956750159000CDE064
:1022B900A852B8000495535002C200740B9000450F
:1022C900F0E567C39464501D900113E0600D90011F
:1022D90013E0A852B80006955340028008C2007462
:1022E9000B900045F0A20040037536059000FCE014
:1022F900B401149000FDE0A852B8000495535007AA
:10230900E55FC39560400280089000A5E0F536803E
:102319003A900084E0B40306A229B3B34002802BAB
:102329009007C4E0C39405A852B800049553500C13
:102339009000A5E0F536740C900045F09007C4E0D4
:10234900A852B8000495535002C20085366C90001B
:1023590076E02536FE900044E075F01E84FC7F008F
:10236900EE2CF53622900044E075F00584FF7E00DE
:102379008F37900044E075F00584ADF07C008D3A0C
:10238900753F05755A03755BD69000C7E01475F063
:102399000584FF7E00E537BE00039F5005120D6AD4
:1023A900800BE53790044C126755E0F537E5379017
:1023B90007C3F09007C3E0FE9000B6E0C39E500843
:1023C9009000B6E09007C3F022E56775F00A84FF34
:1023D9007E0090057612674AE0F546E546D3946497
:1023E9004010E546C3946475F00F84FF7E008F4664
:1023F9008003754600900099E02546F54622900035
:10240900B1E0C3940350269007B0E0FEA3E0FF7447
:1024190004120039E55F126723740F8E048F05FFDC
:102429001267139007AEECF0A3EDF080249007B08B
:10243900E0FEA3E0FF7404120039E561126723741A
:102449000F8E048F05FF1267139007AEECF0A3ED12
:10245900F090008CE0B40262E56AC3944175F0051E
:1024690084FF7E008F37E56A75F00584ADF07C0046
:102479008D3A753F05755A06755B14E537C3941790
:102489005005120D6A800690069DE0F5379007AE5B
:10249900E0FEA3E0FF740A8E048F05FF126713E5BF
:1024A900378C068D07126723740A8E048F05FF1275
:1024B90067139007AEECF0A3EDF09007AEE0FEA332
:1024C900E0FF9007B4E0FCA3E0FDEDD39FEC9E4054
:1024D9000F9007B4E0F8A3E09007AEC8F0A3C8F0E6
:1024E900229006BDE090386BF8282873804C8553FC
:1024F9007380479000C9E0855FF0A4FFAEF07408CF
:102509001200398F738033856173802E85677380DC
:10251900298568738024856973801F856A73801A89
:10252900856B7380158566738010856573800B854F
:0A2539006C738006900016E0F57345
:10386B000224F50224F70224FC022510022515027E
:10387B00251A02251F02252402252902252E0225A1
:07388B003302253802253D40
:102543009006BEE0FE9006BFE0D39E404B9006BDD2
:10255300E0B404189006BFE0C395735002D22A90EA
:1025630006BEE0D395734002C22A802A9006BEE0DD
:10257300C3957350099006BFE0D395735002800250
:10258300D22A9006BEE0D3957350099006BFE0C3EC
:1025930095735002C22A802A9006BEE0D3957340F9
:1025A300099006BFE0C3957340028002C22A9006D9
:1025B300BEE0C3957340099006BFE0D39573400214
:1025C300D22A229006C1E0903892F8282873804CD2
:1025D30085537380479000C9E0855FF0A4FFAEF098
:1025E30074081200398F738033856173802E856779
:1025F3007380298568738024856973801F856A7356
:10260300801A856B7380158566738010856573806A
:0C2613000B856C738006900016E0F573D8
:103892000225D10225D30225D80225EC0225F10208
:1038A20025F60225FB02260002260502260A02262A
:0738B2000F02261402261983
:10261F009006C2E0FE9006C3E0D39E405F9006C1D5
:10262F00E0B404189006C3E0C395735002D22B9008
:10263F0006C2E0D395734002C22B803E9006C2E0E3
:10264F00C3957350099006C3E0D39573500280026F
:10265F00D22B9006C2E0D3957350099006C3E0C306
:10266F0095735002C22B9006C1E0B401099000D5BA
:10267F00E0D3956150028002C22B802A9006C2E0FF
:10268F00D3957340099006C3E0C39573400280024F
:10269F00C22B9006C2E0C3957340099006C3E0D3E6
:1026AF0095734002D22B229006C5E09038B9F828D6
:1026BF002873804C85537380479000C9E0855FF085
:1026CF00A4FFAEF074081200398F738033856173E5
:1026DF00802E856773802985687380248569738050
:1026EF001F856A73801A856B7380158566738010DA
:1026FF00856573800B856C738006900016E0F5730B
:1038B9000226C10226C30226C80226DC0226E1022C
:1038C90026E60226EB0226F00226F50226FA022651
:0738D900FF0227040227098A
:10270F009006C6E0FE9006C7E0D39E404B9006C5EC
:10271F00E0B404189006C7E0C395735002D22C9012
:10272F0006C6E0D395734002C22C802A9006C6E0FD
:10273F00C3957350099006C7E0D39573500280027A
:10274F00D22C9006C6E0D3957350099006C7E0C30C
:10275F0095735002C22C802A9006C6E0D395734021
:10276F00099006C7E0C3957340028002C22C900601
:10277F00C6E0C3957340099006C7E0D39573400236
:10278F00D22C229006C9E09038E0F8282873804CAC
:10279F0085537380479000C9E0855FF0A4FFAEF0CA
:1027AF0074081200398F738033856173802E8567AB
:1027BF007380298568738024856973801F856A7388
:1027CF00801A856B7380158566738010856573809D
:0C27DF000B856C738006900016E0F5730B
:1038E00002279D02279F0227A40227B80227BD02B4
:1038F00027C20227C70227CC0227D10227D60227D8
:07390000DB0227E00227E5CE
:1027EB009006CAE0FE9006CBE0D39E404B9006C904
:1027FB00E0B404189006CBE0C395735002D22D9031
:10280B0006CAE0D395734002C22D802A9006CAE017
:10281B00C3957350099006CBE0D395735002800299
:10282B00D22D9006CAE0D3957350099006CBE0C326
:10283B0095735002C22D802A9006CAE0D39573403F
:10284B00099006CBE0C3957340028002C22D90061F
:10285B00CAE0C3957340099006CBE0D39573400251
:10286B00D22D229006CDE0903907F8282873804CA2
:10287B0085537380479000C9E0855FF0A4FFAEF0ED
:10288B0074081200398F738033856173802E8567CE
:10289B007380298568738024856973801F856A73AB
:1028AB00801A856B738015856673801085657380C0
:0C28BB000B856C738006900016E0F5732E
:1039070002287902287B022880022894022899023B
:10391700289E0228A30228A80228AD0228B202285E
:07392700B70228BC0228C111
:1028C7009006CEE0FE9006CFE0D39E404B9006CD1B
:1028D700E0B404189006CFE0C395735002D22E904F
:1028E70006CEE0D395734002C22E802A9006CEE032
:1028F700C3957350099006CFE0D3957350028002B9
:10290700D22E9006CEE0D3957350099006CFE0C340
:1029170095735002C22E802A9006CEE0D39573405D
:10292700099006CFE0C3957340028002C22E90063D
:10293700CEE0C3957340099006CFE0D3957340026C
:10294700D22E229006D1E090392EF8282873804C99
:1029570085537380479000C9E0855FF0A4FFAEF010
:1029670074081200398F738033856173802E8567F1
:102977007380298568738024856973801F856A73CE
:10298700801A856B738015856673801085657380E3
:0C2997000B856C738006900016E0F57351
:10392E0002295502295702295C02297002297502C3
:10393E00297A02297F02298402298902298E0229E5
:07394E009302299802299D54
:1029A3009006D2E0FE9006D3E0D39E404B9006D132
:1029B300E0B404189006D3E0C395735002D22F906D
:1029C30006D2E0D395734002C22F802A9006D2E04C
:1029D300C3957350099006D3E0D3957350028002D8
:1029E300D22F9006D2E0D3957350099006D3E0C35B
:1029F30095735002C22F802A9006D2E0D39573407C
:102A0300099006D3E0C3957340028002C22F90065B
:102A1300D2E0C3957340099006D3E0D39573400287
:102A2300D22F229006D5E0903955F8282873804C90
:102A330085537380479000C9E0855FF0A4FFAEF033
:102A430074081200398F738033856173802E856714
:102A53007380298568738024856973801F856A73F1
:102A6300801A856B73801585667380108565738006
:0C2A73000B856C738006900016E0F57374
:10395500022A31022A33022A38022A4C022A51024B
:103965002A56022A5B022A60022A65022A6A022A6C
:073975006F022A74022A7997
:102A7F009006D6E0FE9006D7E0D39E404B9006D549
:102A8F00E0B404189006D7E0C395735002D230908B
:102A9F0006D6E0D395734002C230802A9006D6E066
:102AAF00C3957350099006D7E0D3957350028002F7
:102ABF00D2309006D6E0D3957350099006D7E0C375
:102ACF0095735002C230802A9006D6E0D39573409A
:102ADF00099006D7E0C3957340028002C23090067A
:102AEF00D6E0C3957340099006D7E0D395734002A3
:102AFF00D230229006D9E090397CF8282873804C88
:102B0F0085537380479000C9E0855FF0A4FFAEF056
:102B1F0074081200398F738033856173802E856737
:102B2F007380298568738024856973801F856A7314
:102B3F00801A856B73801585667380108565738029
:0C2B4F000B856C738006900016E0F57397
:10397C00022B0D022B0F022B14022B28022B2D02D3
:10398C002B32022B37022B3C022B41022B46022BF3
:07399C004B022B50022B55DA
:102B5B009006DAE0FE9006DBE0D39E404B9006D960
:102B6B00E0B404189006DBE0C395735002D23190A9
:102B7B0006DAE0D395734002C231802A9006DAE080
:102B8B00C3957350099006DBE0D395735002800216
:102B9B00D2319006DAE0D3957350099006DBE0C38F
:102BAB0095735002C231802A9006DAE0D3957340B8
:102BBB00099006DBE0C3957340028002C231900698
:102BCB00DAE0C3957340099006DBE0D395734002BE
:102BDB00D231229006DDE09039A3F8282873804C7F
:102BEB0085537380479000C9E0855FF0A4FFAEF07A
:102BFB0074081200398F738033856173802E85675B
:102C0B007380298568738024856973801F856A7337
:102C1B00801A856B7380158566738010856573804C
:0C2C2B000B856C738006900016E0F573BA
:1039A300022BE9022BEB022BF0022C04022C09025E
:1039B3002C0E022C13022C18022C1D022C22022C7A
:0739C30027022C2C022C311D
:102C37009006DEE0FE9006DFE0D39E404B9006DD77
:102C4700E0B404189006DFE0C395735002D23290C7
:102C570006DEE0D395734002C232802A9006DEE09A
:102C6700C3957350099006DFE0D395735002800235
:102C7700D2329006DEE0D3957350099006DFE0C3A9
:102C870095735002C232802A9006DEE0D3957340D6
:102C9700099006DFE0C3957340028002C2329006B6
:102CA700DEE0C3957340099006DFE0D395734002D9
:102CB700D232229006E1E09039CAF8282873804C76
:102CC70085537380479000C9E0855FF0A4FFAEF09D
:102CD70074081200398F738033856173802E85677E
:102CE7007380298568738024856973801F856A735B
:102CF700801A856B73801585667380108565738070
:0C2D07000B856C738006900016E0F573DD
:1039CA00022CC5022CC7022CCC022CE0022CE502E8
:1039DA002CEA022CEF022CF4022CF9022CFE022D06
:0739EA0003022D08022D0D60
:102D13009006E2E0FE9006E3E0D39E404B9006E18E
:102D2300E0B404189006E3E0C395735002D23390E5
:102D330006E2E0D395734002C233802A9006E2E0B4
:102D4300C3957350099006E3E0D395735002800254
:102D5300D2339006E2E0D3957350099006E3E0C3C3
:102D630095735002C233802A9006E2E0D3957340F4
:102D7300099006E3E0C3957340028002C2339006D4
:102D8300E2E0C3957340099006E3E0D395734002F4
:102D9300D23322AE2EAF2F74F5D39F74019E400819
:102DA300782E126777022EB0752F01752E00AE5262
:102DB300AF53E546BE000DD39F40099000ABE0D36F
:102DC300954740028023754700E546C39553F57345
:102DD3009000AEE0D395454008E5452573F5458061
:102DE300069000AEE0F54580020547900087E0D3EA
:102DF3009561401CE55FC395604015AE52AF53E546
:102E030046BE00039F50099000ACE0D395484002B2
:102E1300806E9007C7E0A852B8000495535003751D
:102E23004A009007C7E0A852B8000BD39553400659
:102E3300E5539007C7F0E54A7041E553C39546F55E
:102E430073E573D3940540037573059000ADE0C338
:102E530095455007E573C3954540028009E545C391
:102E63009573F54580069000ADE0F5459000ADE023
:102E7300D3954540069000ADE0F5457548008002C6
:102E83000548E54A7016900087E0C39561500DE54B
:102E9300462405A852B8000695534002800F9000BF
:102EA3009AE0F545754A0174789007C7F022AE2E73
:102EB300AF2F74E9D39F74039E4008782E1267776F
:102EC30002304F752F01752E00754532A234402A0A
:102ED30075451990009AE075F002A4FFAEF0E5473E
:102EE300BE0006D39F4002D2340547754A03747867
:102EF3009007C7F075490002303EAE52AF53E54626
:102F03006F4E700302303EE546BE000DD39F40096D
:102F13009000ABE0D395474002800F754700E54A28
:102F2300C394035003754519800DE546C39553F5C6
:102F330073E5472573F547900087E0D39561400E0D
:102F43009007C7E0A852B80007D395534002800CFE
:102F5300054990009AE0B54903754A00E54AB40370
:102F630006A20DB3B34002800A0549E549B43C0308
:102F7300754A02E54AB402299007C7E0A852B8008F
:102F83000ED395534009E5539007C7F07549009058
:102F93000087E0C39561500975490074789007C7AD
:102FA300F0E54A705A900087E0D39561401CE55FD5
:102FB300C395604015AE52AF53E546BE00039F5024
:102FC300099000ACE0D3954840028008754800752D
:102FD300454B8028E553C39546F573E573D39405B4
:102FE3004003757305900087E0D395614008E54879
:102FF3002573F5488006E5482406F548754900E53C
:103003004A7016900087E0C39561500DE54624058C
:10301300A852B80006955340028003754A01E54A59
:10302300B40118754519054990009AE0B54906752C
:103033004A0275490074789007C7F0E54575F00AB0
:10304300A4FFAEF09007B8EEF0A3EFF022E56F9087
:1030530039F1F828287390007FE0700302327790EB
:1030630000B5E0B401028003023192900042E0B562
:103073005E02800302318F7E017F00E5BE1267236B
:10308300E5BD2FFF50010E8E5A8F5B74101267231C
:1030930090006DE08E048F05FF1267139007BCEC60
:1030A300F0A3EDF074FFBC00039D500B74FF900779
:1030B300BCF8E4F0E8A3F0E56B600FE56BC394FEA6
:1030C30050089000DBE06402600280649000C9E075
:1030D300B40B1F9007BCE0FEA3E0FF74E712672365
:1030E300E56B8E048F05FF1267139007BCECF0A30A
:1030F300EDF09000C9E0D3940B40089000B1E06478
:10310300046002802B9007BCE0FEA3E0FF9007BEA3
:10311300E0FCA3E0FDEFD39DEE9C400D12676F90A2
:1031230007BCEEF0A3EFF080079007BCE4F0A3F038
:1031330090007FE0B4021E9007BCE0FEA3E0FF9086
:1031430007C8E02FFF50010E74011200399007BC2D
:10315300EEF0A3EFF09007BCE0FEA3E0FF9007C8FA
:10316300E0BE0008D39F4004D2378002B2379007F5
:10317300BDE09007C8F09000B1E064016006A2379B
:10318300B3B3400280069007BDE0F55F023275D20B
:10319300377E017F00E5BE126723E5BD2FFF500197
:1031A3000E8E5A8F5B741012672390006DE08E04AD
:1031B3008F05FF1267139007BCECF0A3EDF0E56BEE
:1031C300600FE56BC394FE50089000DBE06402607F
:1031D3000280649000C9E0B40B1F9007BCE0FEA31B
:1031E300E0FF74E7126723E56B8E048F05FF126718
:1031F300139007BCECF0A3EDF09000C9E0D3940B5F
:1032030040089000B1E064046002802B9007BCE0AA
:10321300FEA3E0FF9007BEE0FCA3E0FDEFD39DEE2D
:103223009C400D12676F9007BCEEF0A3EFF0800790
:103233009007BCE4F0A3F090007FE0B4021E900777
:10324300BCE0FEA3E0FF9007C8E02FFF50010E741F
:10325300011200399007BCEEF0A3EFF09007BDE038
:103263009007C8F09000B1E0640160069007BDE0EC
:10327300F55F8003755F0090007BE07006756F015A
:1032830002305075BB1802384590007BE070030292
:1032930033FD7E017F00E5BE126723E5BD2FFF509E
:1032A300010E8E5A8F5B9000C1E0B4010F7E0F7F39
:1032B300FFAC5AAD5B12676F8E5A8F5B9000E6E0EE
:1032C300B40245AE5AAF5B90001FE0FCA3E0FDEDF6
:1032D300D39FEC9E400A90001FE55AF0A3E55BF0F4
:1032E300AE5AAF5B900021E0FCA3E0FDEFD39DEE6F
:1032F3009C400A900021E55AF0A3E55BF0AE5AAF7B
:103303005B74041200398F619000E6E0704CAE5A92
:10331300AF5B90001FE0FCA3E0FDEFD39DEE9C406C
:103323000912676F8E5A8F5B8006755B00755A00B2
:10333300AE5AAF5B741012672390006AE08E048F5D
:1033430005FF1267138C5A8D5B74FFBC0009D39D74
:103353004005855B6180037561FE9000B1E0B401B7
:103363000280030233FBA20DB3B3500E900085E03D
:10337300A852B80005D39553500280719000C2E063
:103383008561F0A4FFAEF074648E048F05FF1267AD
:10339300138C5A8D5BE56B6016E56BC394FE500F7F
:1033A3009000DBE0B402089000C9E0640B60028087
:1033B30017AE5AAF5B74E7126723E56B8E048F0574
:1033C300FF1267138C5A8D5BAE5AAF5B9007BCE05C
:1033D300FCA3E0FDEDD39FEC9E4005855B5F800B76
:1033E300A237B340069007BDE0F55F800BA237B369
:1033F30040069007BDE0F55F800375610090007E95
:10340300E07006756F0202305075BB1902384590A3
:10341300007EE070030234B2E55ED39551400302AF
:1034230034B090001DE0FEA3E0FFE56512676790EE
:10343300001DEEF0A3EFF07E017F00E5BE126723CF
:10344300E5BD2FFF50010E8E5A8F5B9000EBE070AD
:1034530013740A12672374518E048F05FF126713C6
:103463008D658019AE5AAF5B740A1267238F048E81
:10347300057E017F95CDCCCD1266118F65E565D3B1
:103483009464400375656490001DE0FEA3E0FFE5CE
:10349300652FFF50010E90001DEEF0A3EFF090009A
:1034A30082E0048E048F05FF1267138D6580037518
:1034B30065329000CEE07006756F0302305075BB25
:1034C300130238459000CEE0604A7E017F00E5BEDE
:1034D300126723E5BD2FFF50010E8E5A8F5B7404D4
:1034E3001200398F669000D0E08566F0A4FDACF041
:1034F3007464FF1267138D669000CFE08566F0A4B5
:10350300FFAEF074FF8E048F05FF126713ED90007A
:1035130069F0800375660090007CE07006756F04A7
:1035230002305075BB1702384590007CE0B40102AD
:1035330080030235C07E017F00E5BE126723E5BD2F
:103543002FFF50010E8E5A8F5B9007C9E0601990D0
:1035530007C9E01490619D12008CE493FC740193FD
:10356300FDEDC39FEC9E400280069007C9E014F076
:103573009007C9E0C394B3501DAE5AAF5B9007C91F
:10358300E00490619D12008CE493FC740193FDEFC1
:10359300C39DEE9C400280069007C9E004F09007AB
:1035A300C9E0FE9000A2E08E0088F0A4FFAEF074A4
:1035B300648E048F05FF1267138D678003756700A0
:1035C30090007DE07006756F0502305075BB1602E2
:1035D300384590007DE0B4010280030236697E0124
:1035E3007F00E5BE126723E5BD2FFF50010E8E5A03
:1035F3008F5B9007CAE060199007CAE014906307D5
:1036030012008CE493FC740193FDEDC39FEC9E4088
:103613000280069007CAE014F09007CAE0C394B38F
:10362300501DAE5AAF5B9007CAE0049063071200C7
:103633008CE493FC740193FDEFC39DEE9C400280E8
:10364300069007CAE004F09007CAE0FE9000A8E0E5
:103653008E0088F0A4FFAEF074648E048F05FF1211
:1036630067138D68800375680075BB1F0238457E3C
:10367300017F00E5BE126723E5BD2FFF50010E8ECB
:103683005A8F5B740912672374E68E048F05FF1249
:1036930067138D6A900084E07006756F07023050DF
:1036A30075BB15023845900084E070030237C47E71
:1036B300017F00E5BE126723E5BD2FFF50010E8E8B
:1036C3005A8F5B74041200398F69900084E0B4014F
:1036D300159000D8E08569F0A4FFAEF074071200DE
:1036E30039EF9007C1F0900084E0B402159000D840
:1036F300E08569F0A4FFAEF07407120039EF90077C
:10370300C0F0900084E0B4030280030237A7900066
:10371300C5E0701CE569C394195002D229E569D349
:1037230094644002C2299000A4E09007C4F080632F
:103733009000A4E070349000D8E08569F0A4FFAE57
:10374300F074FF8E048F05FF126713ED9007C4F02A
:10375300AE52AF53741EBE0006D39F4002D229E57A
:1037630061D394E54002C2298029E569C3940A50D4
:103773000DAE52AF53741EBE0004D39F500280029D
:10378300D229E561D394E54002C2299000A4E090D8
:1037930007C4F09007C4E0C394055006740590076E
:1037A300C4F0C238900084E0B40414E569C39419EA
:1037B3005002D238E569D394324002C238C229801C
:1037C300037569009000DBE07006756F08023050E6
:1037D30075BB14806D9000DBE060567E017F00E5D1
:1037E300BE126723E5BD2FFF50010E8E5A8F5BEF8C
:1037F300D39421EE940E4005756BFF8015AE5AAF3E
:103803005B741012672374E38E048F05FF12671332
:103813008D6BE56B75F00BA4FFAEF09000C9E08EE5
:10382300048F05FF1267139007BEECF0A3EDF08041
:1038330003756B0090007FE0600575BB1A8003750C
:02384300BB18B0
:1039F10002305902328C0234120234C702352C02D1
:0B3A010035D50236720236A90237D814
:05384500056FD2EC222A
:096755002582F582500205832221
:0F008C0025E050020583258250020583F582226C
:1066F200EF2F500205832582F582E5833E2EF58336
:016702002274
:10676700CFC39FFF50011E22C3EF9DFFEE9CFE2269
:086777000806B6000218062214
:0D673100A3E004F07006120049E004F0221D
:0E003900048007C3CE13CECF13CFD5E0F6223E
:10661100BC000FBE0008ED8FF084FFADF022E4FE58
:10662100FF22BE000DEF60FE54F0606F20E7030211
:1066310066C7EAC0E0EBC0E078017A0075F001EED0
:1066410020E710EF25E0FFEE33FE0AC5F023C5F089
:1066510030E7F0EA5407F9096A7A007B0060010823
:10666100C3EC9E40167004ED9F4010ED9FFDEC9E23
:10667100FCE5F0CA4ACA03F5F08005E5F003F5F040
:10668100C3EE13FEEF13FFD9D77908CACBCAD8D00E
:10669100EAFEEBFFD0E0FBD0E0FA22EC8FF084FCC5
:1066A100ED54F045F0C48FF084FEEDC454F045F094
:1066B100C48FF084FDEEC4FE54F02DFFEE540F3C68
:1066C100FEADF07C0022790078008FF0EC7E08208E
:1066D100E70DC3CD33CD33C933C9C833C8DEF08428
:1066E10049F9E5F08FF0BE00E6FD7C00E9FFE8FE28
:0166F1002286
:0E672300F88FF0A4FFE5F0CE88F0A42EFE2241
:10000300EF8DF0A4F9A8F0EF8CF0A428F8EE8DF0B2
:06001300A428FEE9FF2213
:10670300600D782B02670D007830D8FED5E0F822B3
:10671300EEC0E07E00126611EFFDEEFCD0E0FE223B
:0C673E00EEC0E07E00126611D0E0FE22EA
:03001B0002001EC2
:0300530002005652
:03009B00020071EF
:0300000002675E36
:09675E0075817575D0000244C577
:0B674A00E5822FF582E5833EF58322F7
:0A0049000582D5820215831582227C
:10001E00C0E0C0F0C083C082C0D075D0001243FFD4
:0B002E00D0D0D082D083D0F0D0E032E0
:10005600C0E0C0F0C083C082C0D075D00012440298
:10006600D0D0D082D083D0F0D0E032C0E0C0F0C093
:1000760083C082C0D075D000124487D0D0D082D041
:0600860083D0F0D0E0324F
:00000001FF
